:020000040000FA
:1000000008DF012045020000690200006B020000C9
:100010006D0200006F020000710200007302000018
:1000200073020000730200007302000073020000FC
:100030007302000073020000FB0200005143000045
:10004000050700000F070000190700002307000044
:100050002D070000250A00002F0A000049090000B2
:100060004F080000BD080000C7080000D1080000CC
:10007000DB080000EF080000610600006B060000CE
:10008000750600007F060000930A00008509000045
:100090008F09000099090000A3090000AD090000C4
:1000A000B7090000430600004D0600005706000097
:1000B00071090000F1060000370700004107000049
:1000C0004B070000390A000053090000C109000075
:1000D000CB09000059080000BB060000C50600005F
:1000E000E706000045080000890A0000E508000056
:1000F0007F0A0000750A00008906000093060000D0
:100100009D060000A7060000DD0600005507000060
:100110005F070000690700005D0900006709000033
:10012000430A00004D0A0000570A0000610A00005F
:100130006B0A0000630800006D080000D50900008C
:10014000DF090000E9090000F3090000FB060000D8
:10015000210900002B090000770800008108000039
:10016000730700007D070000350900007B090000CF
:1001700087070000910700009B070000A50700000B
:10018000AF070000B9070000C3070000CD0700005B
:10019000D7070000E1070000EB070000F5070000AB
:1001A000FF07000009080000130800001D080000F8
:1001B00027080000310800003F090000B1060000D8
:1001C000CF060000B3080000FD090000070A000088
:1001D000110A00001B0A00008B08000095080000AF
:1001E000F908000039060000030900000D090000AD
:1001F000170900009F080000A90800003B08000044
:10020000DFF80CD000F012F900480047416200000E
:1002100008DF0120EFF3108072B67047EFF3108013
:100220007047EFF3108062B6704730BF704780F3BD
:1002300011887047EFF31180704700000138FDD13D
:1002400070470000DFF83000016841F47001016080
:10025000BFF34F8FDFF82400016821F040410160B7
:10026000BFF36F8F06480047FEE7FEE7FEE7FEE7B5
:10027000FEE7FEE7FEE7000088ED00E034EF00E077
:1002800001020000EFF3098141B1F1EE101A40F8CC
:10029000041D20ED200A29490A6810607047B0EC5F
:1002A000200A02C8E1EE101A25490A68106070475A
:1002B000EFF3108072B6704780F3108870472148C2
:1002C0004FF0FF010170002080F309881E4801688B
:1002D00081F308881D48012101701D484FF08051AD
:1002E000016062B6FEE71A484FF080510160704726
:1002F00017484FF080510160704772B6EFF30980E4
:1003000028B1203880E8F00F0C490968086000B572
:10031000104880475DF804EB0F4810490A780270D6
:10032000064807490A680260106890E8F00F20301C
:1003300080F309884EF0F40E62B670473400002056
:100340003C00002022ED00E0000000202E000020F4
:1003500004ED00E01D3F00002300002024000020E9
:1003600072B6704762B67047EFF3108072B670478E
:1003700080F31088704730BF704720BF7047B0FAD5
:1003800080F0704790FAA0F0B0FA80F0704790FAD1
:10039000A0F0704740EA01039B0703D009E008C9B9
:1003A000121F08C0042AFAD203E011F8013B00F83A
:1003B000013B521EF9D27047D2B201E000F8012B86
:1003C000491EFBD270470022F6E710B513460A46D5
:1003D00004461946FFF7F0FF204610BD421E12F8F2
:1003E000013F002BFBD111F8013B02F8013B002B30
:1003F000F9D1704710B5002200E0521C835C8C5C80
:10040000A34201D1002BF8D1D8B2E1B2401A10BDFD
:1004100030B504460020034600E05B1C934203D243
:10042000E05CCD5C401BF8D030BD0000064C074DB1
:1004300006E0E06840F0010394E8070098471034B4
:10044000AC42F6D3FFF7E0FE98B50000B8B5000067
:1004500070B58C1810F8015B15F0070301D110F886
:10046000013B2A1106D110F8012B03E010F8016BB3
:1004700001F8016B5B1EF9D12B0705D40023521E36
:100480000DD401F8013BFAE710F8013BCB1A921C9E
:1004900003E013F8015B01F8015B521EF9D5A1429C
:1004A000D8D3002070BD000000B585B00320002126
:1004B0004FF48052164BCDE90132CDE903100520EF
:1004C0000346144A0090144803F01EFA032000214A
:1004D0004FF48052114BCDE90132CDE903100620D3
:1004E00003460F4A00900F4803F00EFA0320002144
:1004F0004FF4A0720C4BCDE90132CDE903103B2043
:1005000003460A4A00900A4803F0FEF905B000BD10
:10051000083A0120047A0120F54D0000087A0120F4
:1005200004BA0120F74D000008BA012004BF0120E1
:10053000814D000086B000F04FF800F0D7FA044675
:100540004FF47A70B4FBF0F5284603F015FF00F085
:1005500087FB03F0ADF902F0D9FC02F05BFC164812
:1005600003C8CDE9000115480068059014480068EB
:100570000490144800680390DDE9041204F056FC6E
:1005800004F014FB04F032FCFFF78EFF13E00120AF
:1005900002F0FAFB012002F009FC4FF47A7003F03C
:1005A000C1FC002002F0F0FB002002F0FFFB4FF442
:1005B0007A7003F0B7FCEAE7880100208001002090
:1005C0007C01002078010020704770477047704719
:1005D000704770477047704710B500F05FFA00F041
:1005E000DFFA10BD10B50446702C04D204F11001DE
:1005F000C8B200F03BFB10BD70B50446002600BF3A
:1006000000BFFFF7B1FE064600BF00BF02F0E8FDE5
:1006100000BF00BF3046FFF7ABFE00BF00BF702C2D
:1006200004D2044850F8245005B1A84702F0F2FD66
:1006300070BD0000F02B002010B56920FFF7DCFF33
:1006400010BD10B51920FFF7D7FF10BD10B51A2047
:10065000FFF7D2FF10BD10B51B20FFF7CDFF10BD77
:1006600010B50E20FFF7C8FF10BD10B50F20FFF723
:10067000C3FF10BD10B51020FFF7BEFF10BD10B5B1
:100680001120FFF7B9FF10BD10B52E20FFF7B4FF02
:1006900010BD10B52F20FFF7AFFF10BD10B53020F3
:1006A000FFF7AAFF10BD10B53120FFF7A5FF10BD61
:1006B00010B55F20FFF7A0FF10BD10B52620FFF793
:1006C0009BFF10BD10B52720FFF796FF10BD10B59A
:1006D0006020FFF791FF10BD00BFFEE710B532208C
:1006E000FFF78AFF10BD10B52820FFF785FF10BD6A
:1006F00010B51D20FFF780FF10BD10B54320FFF798
:100700007BFF10BD10B50020FFF776FF10BD10B5C0
:100710000120FFF771FF10BD10B50220FFF76CFF3D
:1007200010BD10B50320FFF767FF10BD10B5042002
:10073000FFF762FF10BD10B51E20FFF75DFF10BD73
:1007400010B51F20FFF758FF10BD10B52020FFF790
:1007500053FF10BD10B53320FFF74EFF10BD10B58D
:100760003420FFF749FF10BD10B53520FFF744FFD7
:1007700010BD10B54820FFF73FFF10BD10B5492050
:10078000FFF73AFF10BD10B54C20FFF735FF10BD45
:1007900010B54D20FFF730FF10BD10B54E20FFF70C
:1007A0002BFF10BD10B54F20FFF726FF10BD10B571
:1007B0005020FFF721FF10BD10B55120FFF71CFF9F
:1007C00010BD10B55220FFF717FF10BD10B5532014
:1007D000FFF712FF10BD10B55420FFF70DFF10BD3D
:1007E00010B55520FFF708FF10BD10B55620FFF7D4
:1007F00003FF10BD10B55720FFF7FEFE10BD10B56A
:100800005820FFF7F9FE10BD10B55920FFF7F4FE90
:1008100010BD10B55A20FFF7EFFE10BD10B55B20DC
:10082000FFF7EAFE10BD10B55C20FFF7E5FE10BD36
:1008300010B55D20FFF7E0FE10BD10B56F20FFF78B
:10084000DBFE10BD10B52920FFF7D6FE10BD10B598
:100850000820FFF7D1FE10BD10B52520FFF7CCFE14
:1008600010BD10B53D20FFF7C7FE10BD10B53E20EE
:10087000FFF7C2FE10BD10B54620FFF7BDFE10BD4C
:1008800010B54720FFF7B8FE10BD10B56620FFF782
:10089000B3FE10BD10B56720FFF7AEFE10BD10B55A
:1008A0006D20FFF7A9FE10BD10B56E20FFF7A4FE66
:1008B00010BD10B56120FFF79FFE10BD10B50920D7
:1008C000FFF79AFE10BD10B50A20FFF795FE10BD88
:1008D00010B50B20FFF790FE10BD10B50C20FFF7F0
:1008E0008BFE10BD10B52B20FFF786FE10BD10B596
:1008F0000D20FFF781FE10BD10B56820FFF77CFECC
:1009000010BD10B56A20FFF777FE10BD10B56B2043
:10091000FFF772FE10BD10B56C20FFF76DFE10BD25
:1009200010B54420FFF768FE10BD10B54520FFF755
:1009300063FE10BD10B54A20FFF75EFE10BD10B576
:100940005E20FFF759FE10BD10B50720FFF754FEDB
:1009500010BD10B52220FFF74FFE10BD10B5362098
:10096000FFF74AFE10BD10B53720FFF745FE10BD5A
:1009700010B51C20FFF740FE10BD10B54B20FFF74F
:100980003BFE10BD10B51320FFF736FE10BD10B5AD
:100990001420FFF731FE10BD10B51520FFF72CFE17
:1009A00010BD10B51620FFF727FE10BD10B517209B
:1009B000FFF722FE10BD10B51820FFF71DFE10BD79
:1009C00010B52320FFF718FE10BD10B52420FFF747
:1009D00013FE10BD10B53F20FFF70EFE10BD10B581
:1009E0004020FFF709FE10BD10B54120FFF704FEBF
:1009F00010BD10B54220FFF7FFFD10BD10B56220FD
:100A0000FFF7FAFD10BD10B56320FFF7F5FD10BD2F
:100A100010B56420FFF7F0FD10BD10B56520FFF79D
:100A2000EBFD10BD10B50520FFF7E6FD10BD10B5BC
:100A30000620FFF7E1FD10BD10B52120FFF7DCFD1A
:100A400010BD10B53820FFF7D7FD10BD10B5392007
:100A5000FFF7D2FD10BD10B53A20FFF7CDFD10BD58
:100A600010B53B20FFF7C8FD10BD10B53C20FFF7C7
:100A7000C3FD10BD10B52D20FFF7BEFD10BD10B594
:100A80002C20FFF7B9FD10BD10B52A20FFF7B4FDEB
:100A900010BD10B51220FFF7AFFD10BD10B500243A
:100AA00004E0E0B2034900F007F8641C702CF8D3AE
:100AB00010BD0000D906000070B504460D460026A2
:100AC000702C10D200BF00BFFFF74EFC064600BFDF
:100AD00000BF054840F8245000BF00BF3046FFF774
:100AE00047FC00BF00BF70BDF02B00202DE9F04394
:100AF000DFF89CC0DCF8B0C0CCF3007CBCF1000F88
:100B00003ED0DFF88CC0DCF860C1CCF38A26DFF879
:100B100080C0DCF860C1CCF30A0303EB9622DFF857
:100B200070C0DCF864C1CCF30424DFF864C0DCF8E6
:100B300064C10CF01F05DFF858C0DCF8B0C0CCF37E
:100B4000036111B1032904D101E0124902E0124905
:100B500000E000BF00BF01FB02F804F1010C05F149
:100B600001090CFB09FCB8FBFCF0DFF824C0DCF841
:100B7000B0C0CCF3090C0CF10107B0FBF7F000E0BA
:100B80000020DFF818C0CCF80000BDE8F0830000BA
:100B900000E00F400024F40040787D017400002044
:100BA0002948C06F20F01C002749C8670846C06F5D
:100BB00040F01000C8672448C0300068234908404E
:100BC0002149C1F8C0002048C030006820490843CE
:100BD0001D49C031086048061B49B03108604FF01C
:100BE0004C70086060201B49086004201649C1F859
:100BF00064011848A0380068144908401249C1F837
:100C0000C0001448A0380068134908430E49C1F8D1
:100C1000C0000846D0F8600140F40000C1F860014F
:100C200000BF0C480830006800F0010080F00100AF
:100C30000028F6D10448B03000680849084302494A
:100C4000C1F8B0007047000000E00F4010FC10FC3D
:100C50008100010060E10F408501850103000090E3
:100C600010B500F0F9F800F0BFF810BD2DE9F04123
:100C700004464FF00008102C6BD2DFE804F0080E99
:100C80000F1014293E090A0B0C11120D135300BF4B
:100C900000BF00BF00BF00BF89E000BF00BF00BFB2
:100CA00000BF00BF83E000BF00BFFFF75DFB8046D1
:100CB00000BF00BF3F48006840F480303D490860F5
:100CC00000BF00BF4046FFF753FB00BF00BF6EE010
:100CD00000BF00BFFFF748FB804600BF00BF35489C
:100CE000006840F400303349086000BF00BF404650
:100CF000FFF73EFB00BF00BF59E000BF00BFFFF79A
:100D000033FB804600BF00BF2A48006840F48020C3
:100D10002849086000BF00BF4046FFF729FB00BF1D
:100D200000BF44E000BF00BFFFF71EFB804600BFCE
:100D300000BF4FF0E020006940F001004FF0E021DB
:100D4000086100BF00BF4046FFF712FB00BF00BFB5
:100D50002DE04FF0E0204068401C102101EB4010D6
:100D6000C7B2BC4222DAA4F11000C11700EBD16176
:100D7000C1F34715C11700EBD1614911A0EB411137
:100D8000CEB200BF00BFFFF7EFFA804600BF00BF42
:100D90000120B040A90001F1E021C1F8000100BF2D
:100DA00000BF4046FFF7E4FA00BF00BF00BF00BF2E
:100DB000BDE8F08124ED00E010B5002400BF00BFC5
:100DC000FFF7D2FA044600BF00BF1021054802F029
:100DD00093F800BF00BF2046FFF7CAFA00BF00BF6C
:100DE00010BD0000E02B002010B5FFF7E5FF10BD9F
:100DF0002DE9F04105460C46002714B900BF00F06C
:100E000029F81DB90A202080BDE8F081102128466C
:100E100003F017FF0646102E15D200BF00BFFFF7E4
:100E2000A3FA074600BF00BF10222946084803F076
:100E3000E5FE00BF00BF3846FFF79AFA00BF00BFCB
:100E40000020208002E04FF47A70208000BFDBE7B2
:100E5000E02B002000BFFEE710B50020024908602B
:100E600000F00AF810BD0000700000200149086081
:100E7000704700007000002010B50A48006840F07C
:100E800080700849086000200749486008460068EB
:100E900040F001000860FFF729FE04462046FFF7F6
:100EA000E5FF10BDFCED00E0001000E010B50220F1
:100EB000FFF7C4F904F028F80B48C46904F00C00EB
:100EC00008B1022010BD094803F01CFF0220FFF703
:100ED000B5F904F019F80448C46904F00C0008B12D
:100EE0000220EFE70020EDE700F00A40005800F094
:100EF00010B50346CC00443418591070040A5470DD
:100F0000040C9470040ED470CC0040341859107145
:100F1000040A547110BD10B5CB004033C3586FF3B1
:100F20000F0314792343547943EA0424CB0040335C
:100F3000C4501378547843EA0423947843EA044372
:100F4000D47843EA0464CB004433C45010BD00009D
:100F500070B5D0F8185C156005680C4E35400D6012
:100F6000D0F8DC4004F480351DB1C4F30D051D60DC
:100F70000AE0056805F480151DB14FF420551D6089
:100F800002E04FF400651D6070BD0000FF7E5F7AD7
:100F900030B504680A4D2C400C4344F4004404600E
:100FA00023B143F48034C0F8DC4005E0D0F8DC40E5
:100FB00024F48034C0F8DC40C0F8182C30BD0000A8
:100FC0000C81A0854268024B1A400A434260704778
:100FD00000F8FE7FF0B50446DDE9055700BFDFF8F5
:100FE00094C0DCF800C00CF0010CBCF1000FF6D18D
:100FF00042EA870C4CF08000202D01D8202B03D929
:1010000040F08070ED08DB08AB4202D140EA0520D9
:1010100007E04FF4000C4CEA052C4CEA434C4CEA38
:101020000000C4F8000CDFF850C0DCF814600020A9
:101030000DE0DFF844C05CF830C08C4506D3DFF823
:1010400038C00CEBC00CDCF8046002E0401C032844
:10105000EFD300BFD4F810C02CF03C0C4CEA060CC7
:10106000C4F810C04FF0FF3CC4F80CC1C4F810C164
:10107000F0BD000000CC0E40D4AE000044F24502AA
:101080000A400AB141F4803142F2BA720A400AB110
:1010900041F4004121F000421AB121F00042C0F8B1
:1010A000142C01F000422AB1D0F8D82F42F00102EE
:1010B000C0F8D82F704744F245020A400AB141F403
:1010C000803142F2BA720A400AB141F4004121F083
:1010D000004232B1D0F81C2C21F000431A43C0F872
:1010E0001C2C01F000422AB1D0F8D42F42F00102AA
:1010F000C0F8D42F7047000010B50246D2F8140C87
:10110000094C204021B1D2F81C4C44F0F04420405E
:1011100011B1D2F8D83F01E0D2F8D03F03F001047A
:101120000CB140F0004010BDFFFF01FC70B505465A
:101130000C46C5F8C44F04F0404060B9134803F0B2
:10114000E1FD00BF114803F0C1FD0028FAD042F2D2
:101150001070FFF773F804F04040B0F1404F06D133
:101160000B48006840F480300949086005E00848F1
:10117000006820F4803006490860064800F042F814
:101180004FF47A70FFF75AF870BD0000003000F09D
:10119000C8CF0E4000C00E40034600BF186900F0E3
:1011A00001000028FAD1186900F03C0040EA8210E2
:1011B00040EAC120401C186100BF186900F001001E
:1011C0000028FAD1586980B2704710B500BF046991
:1011D00004F00104002CFAD14361046904F03C04DA
:1011E00044EA821444EAC124E41C046100BF046997
:1011F00004F00104002CFAD110BD0146C86A00F0C9
:1012000061007047D0F8001C41F00101C0F8001CDB
:1012100000BFD0F8001C01F001010029F9D170478E
:10122000C0F80C1C7047D0F8181C41F00201C0F83F
:10123000181C016841F00401016070470146D1F8B3
:1012400028077047C0F8101C70470021C0F8041C24
:101250007047D0F8181C41F40051C0F8181C016800
:1012600041F008010160704702F001031BB1D0F8A2
:1012700000340B4302E0D0F800348B43C0F8003454
:1012800002F002031BB1D0F820340B4302E0D0F887
:1012900020348B43C0F8203470470000F0B55F4D18
:1012A0002D685F4E35405F4EB5421AD0002416E0DF
:1012B0000125A5400D4085B1D0F8C45F6700032625
:1012C000BE40B543C0F8C45FD0F8C45F6700C2F346
:1012D0004116BE403543C0F8C45F651CECB2082C13
:1012E000E6DB02F001051DB1D0F800550D4302E028
:1012F000D0F800558D43C0F8005502F002051DB12D
:10130000D0F804550D4302E0D0F804558D43C0F8E1
:10131000045502F004051DB1D0F808550D4302E054
:10132000D0F808558D43C0F8085502F008051DB1E6
:10133000D0F818550D4302E0D0F818558D43C0F889
:101340001855364D2D68364E3540364EB5420BD0C9
:1013500002F010051DB1D0F83C550D4302E0D0F865
:101360003C558D43C0F83C5503F001051DB1D0F844
:101370000C550D4302E0D0F80C558D43C0F80C55C8
:1013800003F002051DB1D0F810550D4302E0D0F86E
:1013900010558D43C0F8105503F004051DB1D0F869
:1013A00014550D4302E0D0F814558D43C0F8145580
:1013B00003F008051DB1D0F81C550D4302E0D0F82C
:1013C0001C558D43C0F81C55144D2D68144E3540E6
:1013D000144EB54217D003F400751DB1D0F8445532
:1013E0000D4302E0D0F844558D43C0F8445503F452
:1013F00040751DB1D0F840550D4302E0D0F840557E
:101400008D43C0F840551BB9D0F828550D4302E074
:10141000D0F828558D43C0F82855F0BD00E00F40A6
:101420000000FF700000051010B50146C1F3074031
:101430000F4BDB6E01248440234033B1012303EBC7
:1014400040030C4C54F8230003E04300094C54F8CB
:101450002300C1F30722D0F82C350F249440A34376
:1014600001F00F0494402343C0F82C3510BD000058
:1014700000E00F4084B0000030B504460D46022263
:1014800029462046FFF7F0FE08236622294620461B
:10149000FFF704FF30BD30B504460D460222294651
:1014A0002046FFF7E1FE0923012229462046FFF7E7
:1014B000F5FE30BD30B504460D46022229462046D1
:1014C000FFF7D2FE0823012229462046FFF7E6FE59
:1014D00030BD002303EB8103C250704701464868CA
:1014E00000F0010008B1012070470020FCE74160D6
:1014F000704701468868704781607047016A41F013
:101500001001016270470246516801F0010008B104
:101510000020704701F0120010B101F01C00F8E744
:101520000020F6E770B503460C4616461846FFF74E
:10153000E5FF012E01D10F4A00E00F4A142000FB05
:101540000240401E02EB82018900B0FBF1F0451E13
:10155000DD60D3F8C00F00F0010048B10748204417
:10156000401E0649B0FBF1F0451E45F08000D860F2
:1015700070BD0000801A0600A08601008047370178
:1015800042EA410303607047016A41F020010162B1
:101590000121C0F80418704700B502460B461046FA
:1015A000FFF7F2FFC2F8003800BD10B5044614B9C9
:1015B0004FF0FF3010BDA06908B1E06910B94FF0DD
:1015C000FF30F7E79021204600F01CF8002120466C
:1015D00000F002F80020EDE7F8B504460D460820BB
:1015E0008DF800008DF80150A07D02236A466F211E
:1015F000E769B84746B2002E02DA4FF0FF30F8BD77
:101600000020FCE7F8B504460D4607208DF80000E1
:101610008DF80150A07D02236A466F21E769B84723
:1016200046B2002E02DA4FF0FF30F8BD0020FCE792
:1016300010B5002426E0002004EBC4014A4A02EB66
:101640008101086204EBC40102EB8101486004EBF4
:10165000C40102EB81018860172C01D1104605E01E
:10166000601C00EBC000404901EB800004EBC401AA
:101670003D4A02EB8101C8603C4804EBC40142F8DA
:101680002100641C182CD6D3002039498860C8601A
:10169000002459E0032240F2EC51104605F0E4FA30
:1016A00004EBC401334A02EB810108624FF480402D
:1016B00004EBC40102EB8101486004EBC400114655
:1016C00001EB8000006A18B304EBC40001EB80005A
:1016D000006A406804EBC40102EB8101886004EBFE
:1016E000C400114601EB8000406804EBC40102EB2A
:1016F0008101096A4989084304EBC40102EB8101B5
:1017000048604FF0004004EBC40142F821000AE0B9
:10171000002004EBC401174A02EB8101886004EB4E
:10172000C40142F82100072C01D1124805E0601CD9
:1017300000EBC0000F4901EB800004EBC4010D4A2F
:1017400002EB8101C860641C082CA3D30020084967
:101750008860C86007490848FFF762FD02490648EB
:10176000FFF770FD10BD0000BC2A01200000D04032
:10177000200100201C2E012000C00E40042806D1AC
:101780001949096841F48031174A11602BE0052896
:1017900006D11549096841F40031134A116022E06D
:1017A000062806D11049096841F480210E4A1160CB
:1017B00019E00F2808D14FF0E021096941F002013A
:1017C0004FF0E02211610EE010280CD3A0F11001BF
:1017D00001F01F0201219140A0F110025209034BB8
:1017E00053F822201160704724ED00E0D0B10000D2
:1017F00010B5FEF716FD08B1012010BD0020FCE772
:1018000010B5084803F02CFA00BF064803F05EFA52
:101810000028FAD0FFF74AFB04460CB100BFFEE7F0
:1018200010BD0000005800F02DE9F04104460D46BF
:1018300016461F46082C03DB4FF0FF30BDE8F08151
:1018400000BF04EB4400EC4901EB8000C0780128A4
:10185000F7D004EB440001EB800000790128F0D0C0
:10186000002004EB4401E44A02F8210004EB4400A8
:10187000114601EB8000467004EB440001EB800050
:10188000877004EB440001EB8000856014BBDB48EB
:1018900003F0E6F9DA4803F0E3F9D94803F0E0F998
:1018A000D848FFF7C1FDD848FFF7BEFD0421D7484F
:1018B000FFF700FE0821D548FFF7EDFDA6B9D44893
:1018C000854208D103F056FA804600224146D148AD
:1018D000FFF728FE0CE003F04DFA80460122414656
:1018E000CC48FFF71FFE03E03946CA48FFF754FE15
:1018F000012C33D1C148401C03F0B2F9C048401D4F
:1019000003F0AEF9BE48401D03F0AAF9C248FFF744
:101910008BFDC248FFF788FD0121C148FFF7CAFDD2
:101920000221BF48FFF7B7FDA6B9B948854208D1E3
:1019300003F020FA804600224146BA48FFF7F2FD44
:101940000CE003F017FA804601224146B548FFF744
:10195000E9FD03E03946B348FFF71EFE022C33D100
:10196000A648801C03F07CF9A548093003F078F9FB
:10197000A348093003F074F9AB48FFF755FDAB48B5
:10198000FFF752FD0221AA48FFF794FD0121A84864
:10199000FFF781FDA6B99E48854208D103F0EAF918
:1019A000804600224146A348FFF7BCFD0CE003F04F
:1019B000E1F98046012241469E48FFF7B3FD03E06E
:1019C00039469C48FFF7E8FD032C33D18B48C01CF7
:1019D00003F046F98A48083003F042F98848083095
:1019E00003F03EF99448FFF71FFD9448FFF71CFDF4
:1019F00010219348FFF75EFD20219148FFF74BFD32
:101A0000A6B98348854208D103F0B4F98046002284
:101A100041468C48FFF786FD0CE003F0ABF98046A9
:101A2000012241468748FFF77DFD03E0394685489E
:101A3000FFF7B2FD042C33D17048001D03F010F9FC
:101A40006F48083003F00CF96D48083003F008F9CE
:101A50007D48FFF7E9FC7D48FFF7E6FC4021784828
:101A6000FFF728FD80217648FFF715FDA6B96848E5
:101A7000854208D103F07EF9804600224146744831
:101A8000FFF750FD0CE003F075F980460122414656
:101A90006F48FFF747FD03E039466D48FFF77CFDCF
:101AA000052C31D15548401D03F0DAF8544803F0B5
:101AB000D7F8534803F0D4F86648FFF7B5FC6648FA
:101AC000FFF7B2FC01215148FFF7F4FC02214F4817
:101AD000FFF7E1FCA6B94E48854208D103F04AF968
:101AE0008046002241465D48FFF71CFD0CE003F0F4
:101AF00041F98046012241465848FFF713FD03E0B3
:101B000039465648FFF748FD062C37D13B48801D23
:101B100003F0A6F83A48401E03F0A2F83848401EE9
:101B200003F09EF841F60200FFF77EFC41F602400A
:101B3000FFF77AFC40214FF04020FFF7BBFC8021EB
:101B40004FF04020FFF7A7FCA6B93148854208D1E5
:101B500003F010F98046002241464148FFF7E2FCBD
:101B60000CE003F007F98046012241463C48FFF7AC
:101B7000D9FC03E039463A48FFF70EFD072C33D174
:101B80001E48C01D03F06CF81D48801C03F068F867
:101B90001B48801C03F064F83248FFF745FC3248CC
:101BA000FFF742FC01213148FFF784FC02212F4856
:101BB000FFF771FCA6B91648854208D103F0DAF8A0
:101BC0008046002241462A48FFF7ACFC0CE003F0B7
:101BD000D1F88046012241462548FFF7A3FC03E0E7
:101BE00039462348FFF7D8FC012004EB4401024AA0
:101BF00002F82100002021E6B02D0020002000F096
:101C0000010800F002080100020C01000050004031
:101C1000A086010000000240020006000204060047
:101C2000006002400010024002040A0002000A00A4
:101C300000200640002002400210090002140900A2
:101C4000001006400030024002180900021C090082
:101C500000000C40020001000204010000100C40D2
:101C600000200C400200030002040300007000404A
:101C700000300C402DE9F0470546884617461E46C1
:101C80004FF00009082D03DB4FF0FF30BDE8F0876F
:101C900037B12EB105EB4500FA4911F8200010B913
:101CA0004FF0FF30F2E7FEF703FB8146012005EB22
:101CB0004501F44A02EB8101C87005EB450011466D
:101CC00001EB80004078002878D1002D78D100BF4A
:101CD000ED48FFF703FC0028FAD101224146EA480B
:101CE000FFF74EFC012E29D10721E748FFF7FFFB44
:101CF000E548FFF708FC58B1002005EB4501E14A33
:101D000002EB8101C8704846FEF7D6FAB01EBDE767
:101D100000BFDD48FFF7E2FB0028FAD1DA48FFF701
:101D2000E8FB3870002005EB4501D64A02EB810143
:101D3000C8704846FEF7C0FA0020A7E700243BE041
:101D400024B90B21D048FFF7D2FB0BE0701EA04254
:101D500004D10521CC48FFF7CAFB03E00921CA489A
:101D6000FFF7C5FBC848FFF7CEFBD0B1701EA042FD
:101D70000AD0C548FFF7C7FB00F01000102803D0B9
:101D80000421C148FFF7B3FB002005EB4501BD4A24
:101D900002EB8101C8704846FEF78EFA4FF0FF3023
:101DA00074E700BFB848FFF799FB0028FAD1B6489E
:101DB000FFF79FFB3855641CB442C1D365E3FFE7CE
:101DC000012D78D100BFB148FFF788FB0028FAD178
:101DD00001224146AD48FFF7D3FB012E29D107214F
:101DE000AA48FFF784FBA948FFF78DFB58B10020F4
:101DF00005EB4501A34A02EB8101C8704846FEF796
:101E00005BFAB01E42E700BFA048FFF767FB00285F
:101E1000FAD19E48FFF76DFB3870002005EB4501B5
:101E2000984A02EB8101C8704846FEF745FA002047
:101E30002CE700243BE024B90B219448FFF757FB23
:101E40000BE0701EA04204D105219048FFF74FFB24
:101E500003E009218D48FFF74AFB8C48FFF753FB4D
:101E6000D0B1701EA0420AD08848FFF74CFB00F0AA
:101E70001000102803D004218448FFF738FB00200D
:101E800005EB45017F4A02EB8101C8704846FEF729
:101E900013FA4FF0FF30F9E600BF7C48FFF71EFB56
:101EA0000028FAD17948FFF724FB3855641CB44266
:101EB000C1D3EAE2FFE7022D78D100BF7448FFF7F3
:101EC0000DFB0028FAD1012241467148FFF758FB6B
:101ED000012E29D107216E48FFF709FB6C48FFF757
:101EE00012FB58B1002005EB4501664A02EB810167
:101EF000C8704846FEF7E0F9B01EC7E600BF644868
:101F0000FFF7ECFA0028FAD16148FFF7F2FA3870CF
:101F1000002005EB45015B4A02EB8101C870484691
:101F2000FEF7CAF90020B1E600243BE024B90B21FA
:101F30005748FFF7DCFA0BE0701EA04204D10521E0
:101F40005348FFF7D4FA03E009215148FFF7CFFACD
:101F50004F48FFF7D8FAD0B1701EA0420AD04C48C3
:101F6000FFF7D1FA00F01000102803D004214848F0
:101F7000FFF7BDFA002005EB4501424A02EB810163
:101F8000C8704846FEF798F94FF0FF307EE600BF74
:101F90003F48FFF7A3FA0028FAD13D48FFF7A9FA16
:101FA0003855641CB442C1D36FE2FFE7032D73D1EF
:101FB00000BF3848FFF792FA0028FAD101224146C3
:101FC0003448FFF7DDFA012E29D107213148FFF708
:101FD0008EFA3048FFF797FA58B1002005EB45011B
:101FE000284A02EB8101C8704846FEF765F9B01E29
:101FF0004CE600BF2748FFF771FA0028FAD12548C0
:10200000FFF777FA3870002005EB45011D4A02EB17
:102010008101C8704846FEF74FF9002036E60024DB
:1020200046E024B90B211B48FFF761FA0BE0701E54
:10203000A04204D105211748FFF759FA03E009210E
:102040001448FFF754FA1348FFF75DFA28B3701EDF
:10205000A0420AD00F48FFF756FA00F010001028EF
:1020600003D004210B48FFF742FA002005EB45019D
:10207000044A02EB8101C8704846FEF71DF94FF093
:10208000FF3003E6B02D00200000024000100240A7
:1020900000200240003002400DE000BFFE48FFF784
:1020A0001DFA0028FAD1FC48FFF723FA3855641CC2
:1020B000B442B6D3E9E1042D78D100BFF748FFF769
:1020C0000DFA0028FAD101224146F448FFF758FAE8
:1020D000012E29D10721F148FFF709FAEF48FFF750
:1020E00012FA58B1002005EB4501ED4A02EB8101DF
:1020F000C8704846FEF7E0F8B01EC7E500BFE748E5
:10210000FFF7ECF90028FAD1E448FFF7F2F938704C
:10211000002005EB4501E24A02EB8101C870484608
:10212000FEF7CAF80020B1E500243BE024B90B21FA
:10213000DA48FFF7DCF90BE0701EA04204D105215C
:10214000D648FFF7D4F903E00921D448FFF7CFF9C7
:10215000D248FFF7D8F9D0B1701EA0420AD0CF48BC
:10216000FFF7D1F900F01000102803D00421CB486C
:10217000FFF7BDF9002005EB4501C94A02EB8101DB
:10218000C8704846FEF798F84FF0FF307EE500BF74
:10219000C248FFF7A3F90028FAD1C048FFF7A9F910
:1021A0003855641CB442C1D36FE1FFE7052D78D1E7
:1021B00000BFBC48FFF792F90028FAD1012241463E
:1021C000B848FFF7DDF9012E29D10721B548FFF7FF
:1021D0008EF9B448FFF797F958B1002005EB450197
:1021E000AF4A02EB8101C8704846FEF765F8B01EA1
:1021F0004CE500BFAB48FFF771F90028FAD1A948B8
:10220000FFF777F93870002005EB4501A44A02EB8F
:102210008101C8704846FEF74FF8002036E50024DB
:102220003BE024B90B219F48FFF761F90BE0701EDA
:10223000A04204D105219B48FFF759F903E0092189
:102240009848FFF754F99748FFF75DF9D0B1701E31
:10225000A0420AD09348FFF756F900F0100010286A
:1022600003D004218F48FFF742F9002005EB450118
:102270008B4A02EB8101C8704846FEF71DF84FF00B
:10228000FF3003E500BF8748FFF728F90028FAD19F
:102290008448FFF72EF93855641CB442C1D3F4E0EA
:1022A000FFE7062D78D100BF7F48FFF717F9002818
:1022B000FAD1012241467C48FFF762F9012E29D16B
:1022C00007217948FFF713F97748FFF71CF958B150
:1022D000002005EB4501724A02EB8101C8704846B7
:1022E000FDF7EAFFB01ED1E400BF6F48FFF7F6F834
:1022F0000028FAD16C48FFF7FCF83870002005EB95
:102300004501674A02EB8101C8704846FDF7D4FFDA
:102310000020BBE400243BE024B90B216248FFF716
:10232000E6F80BE0701EA04204D105215E48FFF7DD
:10233000DEF803E009215C48FFF7D9F85A48FFF7B7
:10234000E2F8D0B1701EA0420AD05748FFF7DBF880
:1023500000F01000102803D004215348FFF7C7F8FD
:10236000002005EB45014E4A02EB8101C87048464A
:10237000FDF7A2FF4FF0FF3088E400BF4A48FFF7A7
:10238000ADF80028FAD14848FFF7B3F83855641C77
:10239000B442C1D379E0FFE7072D76D100BF4348AF
:1023A000FFF79CF80028FAD1012241463F48FFF789
:1023B000E7F8012E29D107213C48FFF798F83B4860
:1023C000FFF7A1F858B1002005EB4501344A02EBB4
:1023D0008101C8704846FDF76FFFB01E56E400BF8C
:1023E0003248FFF77BF80028FAD13048FFF781F830
:1023F0003870002005EB4501294A02EB8101C870C5
:102400004846FDF759FF002040E400243BE024B992
:102410000B212648FFF76BF80BE0701EA04204D199
:1024200005212248FFF763F803E009211F48FFF761
:102430005EF81E48FFF767F8D0B1701EA0420AD0C0
:102440001A48FFF760F800F01000102803D00421AC
:102450001648FFF74CF8002005EB4501104A02EB47
:102460008101C8704846FDF727FF4FF0FF300DE4AB
:1024700000BF0E48FFF732F80028FAD10B48FFF7EB
:1024800038F83855641CB442C1D3002005EB45012F
:10249000034A02EB81010BE00030024000000C40D7
:1024A000B02D002000100C4000200C4000300C40EB
:1024B000C8704846FDF700FF002028E42DE9F047EA
:1024C0000546884616461F464FF00009082D03DBD7
:1024D0004FF0FF30BDE8F08736B12FB105EB450076
:1024E000F74911F8200010B94FF0FF30F2E7FDF77F
:1024F000DFFE8146012005EB4501F14A02EB810137
:10250000087105EB4500114601EB8000407800287A
:1025100076D1002D75D100BFEA48FEF7DFFF002815
:10252000FAD100224146E748FFF72AF8012F28D1C7
:102530003178E448FEF7E0FF0721E248FEF7D7FFD5
:10254000E048FEF7E0FF58B1002005EB4501DC4A0A
:1025500002EB810108714846FDF7AEFEB81EB9E7EF
:1025600000BFD848FEF7BAFF0028FAD105EB4501B5
:10257000D34A02EB810108714846FDF79DFE002019
:10258000A8E7002445E044B9315DCE48FEF7B4FF2A
:102590000321CC48FEF7ABFF13E0781EA04208D120
:1025A000315DC848FEF7A8FF0521C648FEF79FFF2A
:1025B00007E0315DC348FEF79FFF0121C148FEF7E8
:1025C00096FFC048FEF79FFFE0B1781EA0420AD0F8
:1025D000BC48FEF798FF00F01000102803D004213B
:1025E000B848FEF784FF002005EB4501B44A02EB32
:1025F000810108714846FDF75FFE4FF0FF3069E743
:102600001CE209E000BFAF48FEF768FF0028FAD1DE
:10261000641CBC42B7D3A5E3012D7FD100BFAA48FB
:10262000FEF75CFF0028FAD100224146A648FEF7DB
:10263000A7FF012F28D13178A348FEF75DFF0721BE
:10264000A148FEF754FFA048FEF75DFF58B10020F7
:1026500005EB45019A4A02EB810108714846FDF7F6
:102660002BFEB81E36E700BF9748FEF737FF00285D
:10267000FAD105EB4501924A02EB81010871484607
:10268000FDF71AFE002025E7002444E044B9315D3F
:102690008D48FEF731FF03218B48FEF728FF13E03A
:1026A000781EA04208D1315D8748FEF725FF05213D
:1026B0008548FEF71CFF07E0315D8348FEF71CFFED
:1026C00001218148FEF713FF7F48FEF71CFFD8B1B8
:1026D000781EA0420AD07C48FEF715FF00F01000DB
:1026E000102803D004217848FEF701FF002005EBF5
:1026F0004501734A02EB810108714846FDF7DCFD94
:102700004FF0FF30E6E609E000BF6F48FEF7E6FE57
:102710000028FAD1641CBC42B8D323E3022D7FD138
:1027200000BF6A48FEF7DAFE0028FAD100224146CF
:102730006648FEF725FF012F28D131786348FEF760
:10274000DBFE07216148FEF7D2FE6048FEF7DBFEA4
:1027500058B1002005EB4501594A02EB810108718F
:102760004846FDF7A9FDB81EB4E600BF5748FEF77E
:10277000B5FE0028FAD105EB4501514A02EB810173
:1027800008714846FDF798FD0020A3E6002444E0C8
:1027900044B9315D4D48FEF7AFFE03214B48FEF7CB
:1027A000A6FE13E0781EA04208D1315D4748FEF72F
:1027B000A3FE05214548FEF79AFE07E0315D434838
:1027C000FEF79AFE01214148FEF791FE3F48FEF7D1
:1027D0009AFED8B1781EA0420AD03C48FEF793FE7C
:1027E00000F01000102803D004213848FEF77FFEC7
:1027F000002005EB4501324A02EB81010871484691
:10280000FDF75AFD4FF0FF3064E609E000BF2F48A6
:10281000FEF764FE0028FAD1641CBC42B8D3A1E2E2
:10282000032D7CD100BF2A48FEF758FE0028FAD1BC
:10283000002241462648FEF7A3FE012F28D1317819
:102840002348FEF759FE07212148FEF750FE204895
:10285000FEF759FE58B1002005EB4501184A02EB7E
:10286000810108714846FDF727FDB81E32E600BF1A
:102870001748FEF733FE0028FAD105EB4501104A50
:1028800002EB810108714846FDF716FD002021E6A4
:1028900000244FE044B9315D0D48FEF72DFE0321C1
:1028A0000B48FEF724FE1DE0781EA04212D1315DD8
:1028B0000748FEF721FE05210548FEF718FE11E046
:1028C000B02D002000000240001002400020024015
:1028D00000300240315DF848FEF70EFE0121F64857
:1028E000FEF705FEF448FEF70EFEE0B1781EA042AA
:1028F0000AD0F148FEF707FE00F01000102803D0C0
:102900000421ED48FEF7F3FD002005EB4501EB4AFD
:1029100002EB810108714846FDF7CEFC00E00CE0B7
:102920004FF0FF30D6E500BFE348FEF7D7FD0028A3
:10293000FAD1641CBC42ADD314E2042D7FD100BF98
:10294000DF48FEF7CBFD0028FAD100224146DC48E3
:10295000FEF716FE012F28D13178D948FEF7CCFDBD
:102960000721D748FEF7C3FDD548FEF7CCFD58B187
:10297000002005EB4501D14A02EB81010871484670
:10298000FDF79AFCB81EA5E500BFCD48FEF7A6FDF1
:102990000028FAD105EB4501C84A02EB8101087114
:1029A0004846FDF789FC002094E5002444E044B942
:1029B000315DC348FEF7A0FD0321C148FEF797FD36
:1029C00013E0781EA04208D1315DBD48FEF794FDAA
:1029D0000521BB48FEF78BFD07E0315DB848FEF7E7
:1029E0008BFD0121B648FEF782FDB548FEF78BFD51
:1029F000D8B1781EA0420AD0B148FEF784FD00F09D
:102A00001000102803D00421AD48FEF770FD00200F
:102A100005EB4501A94A02EB810108714846FDF723
:102A20004BFC4FF0FF3055E509E000BFA448FEF72E
:102A300055FD0028FAD1641CBC42B8D392E1052DA3
:102A40007FD100BF9F48FEF749FD0028FAD1002240
:102A500041469C48FEF794FD012F28D131789948D2
:102A6000FEF74AFD07219748FEF741FD9548FEF71E
:102A70004AFD58B1002005EB4501904A02EB810167
:102A800008714846FDF718FCB81E23E500BF8D48C5
:102A9000FEF724FD0028FAD105EB4501874A02EB39
:102AA000810108714846FDF707FC002012E500246B
:102AB00044E044B9315D8348FEF71EFD032181489F
:102AC000FEF715FD13E0781EA04208D1315D7D4868
:102AD000FEF712FD05217B48FEF709FD07E0315D99
:102AE0007848FEF709FD01217648FEF700FD75489C
:102AF000FEF709FDD8B1781EA0420AD07148FEF752
:102B000002FD00F01000102803D004216D48FEF7EC
:102B1000EEFC002005EB4501684A02EB81010871DB
:102B20004846FDF7C9FB4FF0FF30D3E409E000BF92
:102B30006448FEF7D3FC0028FAD1641CBC42B8D329
:102B400010E1062D7FD100BF5F48FEF7C7FC0028CB
:102B5000FAD1002241465C48FEF712FD012F28D130
:102B600031785948FEF7C8FC07215748FEF7BFFCEB
:102B70005548FEF7C8FC58B1002005EB45014F4A07
:102B800002EB810108714846FDF796FBB81EA1E4EF
:102B900000BF4D48FEF7A2FC0028FAD105EB450125
:102BA000464A02EB810108714846FDF785FB00208B
:102BB00090E4002444E044B9315D4348FEF79CFCB6
:102BC00003214148FEF793FC13E0781EA04208D190
:102BD000315D3D48FEF790FC05213B48FEF787FC40
:102BE00007E0315D3848FEF787FC01213648FEF7E3
:102BF0007EFC3548FEF787FCD8B1781EA0420AD08B
:102C00003148FEF780FC00F01000102803D00421AA
:102C10002D48FEF76CFC002005EB4501274A02EB2E
:102C2000810108714846FDF747FB4FF0FF3051E442
:102C300009E000BF2448FEF751FC0028FAD1641CCB
:102C4000BC42B8D38EE0072D7DD100BF1F48FEF7F0
:102C500045FC0028FAD1002241461C48FEF790FCB2
:102C6000012F35D131781948FEF746FC0721174866
:102C7000FEF73DFC1548FEF746FC58B1002005EB79
:102C800045010E4A02EB810108714846FDF714FB2D
:102C9000B81E1FE400BF0D48FEF720FC0028FAD143
:102CA00005EB4501054A02EB810108714846FDF735
:102CB00003FB00200EE4000000300240B02D002095
:102CC00000000C4000100C4000200C4000300C4074
:102CD000002445E044B9315D2848FEF70DFC03218E
:102CE0002648FEF704FC13E0781EA04208D1315DAF
:102CF0002248FEF701FC05212048FEF7F8FB07E01B
:102D0000315D1E48FEF7F8FB01211C48FEF7EFFB82
:102D10001A48FEF7F8FBE0B1781EA0420AD0174827
:102D2000FEF7F1FB00F01000102803D00421134837
:102D3000FEF7DDFB002005EB4501114A02EB8101A6
:102D40000871484600E00DE0FDF7B6FA4FF0FF309D
:102D500005E400BF0948FEF7C1FB0028FAD1641C56
:102D6000BC42B7D3002005EB4501054A02EB8101C7
:102D700008714846FDF7A0FA002040E400300C40FE
:102D8000B02D00207047000010B504462CB9012278
:102D900011460548FEF79DFB04E0FE220121024892
:102DA000FEF797FB10BD00000070004010B5044610
:102DB0002CB9022211460548FEF78BFB04E0FD22E8
:102DC00002210248FEF785FB10BD000000700040A4
:102DD00010B50E4801F044FF012211460C48FEF7E1
:102DE00043FA0823012211460948FEF757FA07481B
:102DF00001F036FF012202210548FEF735FA0823CB
:102E0000012202210248FEF749FA10BD030800F032
:102E10000070004010B5FFF7B5FFFFF7D9FFFEF7D0
:102E2000E7FCFEF7EDFC10BD10B54FF0804001F05F
:102E3000F7FF01F09FFF044621464FF0804001F06C
:102E4000E7FF4FF0804001F0DFFF10BD0020014997
:102E5000087070477800002010B54FF0704001F006
:102E6000FFFE2220FEF78AFC4FF0804001F0D8FFE1
:102E700001F080FF044621464FF0804001F0C8FF7A
:102E80004FF0804001F0C6FF4FF0804001F0BCFFE2
:102E900005491220FDF710FE1220FDF7A3FB4FF0AD
:102EA000804001F0A9FF10BDAD2E000010B500F06C
:102EB00097F90C480078401C0A49087008460078C9
:102EC0001E2802DD0120084908700748007828B94B
:102ED0004FF0804001F095FFFFF7A6FF00F09AF950
:102EE00010BD000078000020790000200120014979
:102EF000087070477900002030B505460C46224620
:102F00000021284600F026F830BD00000D480E498B
:102F100001600146416000218160C1600161416141
:102F20008161C16101620163C162416207498163DC
:102F3000C1634FF48061016441640146044A116039
:102F4000704700009827002048454150E0270020A6
:102F50006C0000202DE9F04103460C4617460FB9DE
:102F6000BDE8F08103B9FBE70025002202E02D0255
:102F70002543521C042AFAD3384603F0030C1946A1
:102F8000BCF1000F08D0624603E001F8014B401E7F
:102F9000521C08B1042AF8D30E4601E020C6001FD7
:102FA0000428FBD2314602E001F8014B401E002804
:102FB000FAD100BFD4E700001D481E481E481F4834
:102FC0001F482048204821482148224822482348B9
:102FD0002348244824482548254826482648274889
:102FE000274828482848294829482A482A482B4859
:102FF0002B482C482C482D482D482E482E482F4829
:103000002F483048304831483148324832483348F8
:1030100033483448344835483548364836483748C8
:103020003748384838483948394800BF70470000A9
:1030300020B2000024B200002AB200002CB200002E
:1030400028B200002EB2000030B2000032B2000000
:1030500034B2000036B2000038B200003AB20000CC
:103060003CB200003EB2000040B2000042B200009C
:1030700044B2000046B2000048B200004AB200006C
:103080004CB200004EB2000050B2000052B200003C
:1030900054B2000056B2000058B200005AB200000C
:1030A0005CB200005EB2000060B2000062B20000DC
:1030B00064B2000066B2000068B200006AB20000AC
:1030C0006CB200006EB2000070B2000072B200007C
:1030D00076B2000078B200007AB200007CB2000044
:1030E000D82200205827002080B2000082B20000C1
:1030F00084B2000086B2000088B200008AB20000EC
:103100008CB200008EB2000090B200007EB20000CF
:1031100092B200002DE9F04105460E461446002704
:103120001148007818B112202070BDE8F08128788D
:10313000012808D0022807D0032802D0042804D18F
:1031400000E000BF00BF00BF02E001202070ECE7FC
:1031500000BFFDF7ADF807466E613846FDF7ACF8E5
:103160000020207000BFE0E72100002010B500F033
:1031700019F801F051FA01F07DFA01F09DFA01F021
:103180001BFA01F0DBF901F031FB01F05BFB01F010
:10319000D3FA01F0F9FA00F0A1FF00F01FF8FFF7F1
:1031A0000BFF10BD0948802102E0491E002204C027
:1031B0000029FAD1064A074B1A601A46126822F013
:1031C00007021A600022044B1A8070479001002009
:1031D0009003002000000020040000207047000041
:1031E00010B50024FDF764F804460848007801286B
:1031F00008D107480078FF2804D205480078401C11
:10320000034908702046FDF757F810BD2E00002036
:103210002100002010B500241A480078012830D180
:10322000FDF746F804461848007820B116480078A3
:10323000401E1549087014480078F8B91348007802
:10324000E0B901F061FB12481249097850F82100F9
:10325000114908600F4800781049097888420DD05C
:103260000D480068C06B401C0B490968C8630C48D6
:103270000068401C0A490860FDF73AF82046FDF74F
:103280001BF810BD2E00002021000020220000208D
:10329000180E0020240000203C0000202300002005
:1032A000080000202DE9FC5F05460F4691469A462E
:1032B00000200090FCF7FCFF0090184804680068AC
:1032C00020B1164800684068144908600098FCF76F
:1032D000F3FF2CB95A208AF800000020BDE8FC9FBB
:1032E000A8462E46781E01904FF0000B05E04E4494
:1032F000C8F80060B0460BF1010B01988345F6D386
:103300000020C8F80000256065602761E760C4F808
:1033100008908AF800002046E0E7000048000020FE
:103320002DE9F04104460D460027FCF7C1FF074692
:10333000206968B16668306860602069401E20615D
:103340003846FCF7B9FF002028703046BDE8F08110
:103350003846FCF7B1FF5D2028700020F6E770B515
:1033600004460D460026FCF7A3FF0646D4E90310E9
:10337000884204D33046FCF79FFF5E2070BD606832
:10338000286065602069401C20613046FCF794FF8E
:103390000020F3E72DE9F04106460F464FF0000804
:1033A0002048007810B10020BDE8F081FCF780FFD4
:1033B00080461D480468006820B11B4800684068CA
:1033C000194908604046FCF777FFFCB1FCF770FF35
:1033D000804616480568D5B1006800681349086042
:1033E0004046FCF769FF6E6006EB8700A860EE6060
:1033F0002E61AF820020E882022020700020208110
:1034000065600BA06061204601F08AF808E006487C
:1034100000686060044804604046FCF74DFF0024EB
:103420002046C1E7210000200C0000204C000020B5
:103430003F0000002DE9F0470746884615464FF04B
:1034400000093878022804D0012028700020BDE847
:10345000F0873E48007818B1022028700020F6E777
:103460003B48007818B10D2028700020EFE7FCF7EA
:103470001FFF81467C68E08A98B12169081D2061A0
:103480000E68E08A401EE082A1682069884201D16E
:10349000606820614846FCF70FFF00202870304626
:1034A000D5E72C48006890F8340040F00400294922
:1034B000096881F8340000202649096881F8350040
:1034C00024480068C0F83080384600F0EBFF4846DA
:1034D000FCF7F2FE01F0DEF9FCF7EAFE81461D483A
:1034E000006890F8350020B101280DD002280AD1DB
:1034F00005E018480068466A002028700DE00026A4
:103500000E20287009E000BF39461248006800F01C
:1035100095FF00260A20287000BF00BF00200D493B
:10352000096881F834000B49096881F835000949B8
:103530000968C8610749096808620649096848625C
:103540004846FCF7B9FE304681E700002100002024
:1035500022000020340000202DE9F04105460E46EF
:1035600000272878022802D00120BDE8F081FCF76E
:103570009FFE0746A87A60B1002304223146284600
:1035800000F014FF3846FCF797FE01F083F90020A5
:10359000EBE76C68E08AA18A884204DB3846FCF7D6
:1035A0008BFE1E20E1E7E168081DE0600E60E08A06
:1035B000401CE082D4E90210884201D16068E060DA
:1035C0003846FCF779FE0020CFE72DE9F0470546A5
:1035D0000C464FF0000A2878022802D00120BDE8EE
:1035E000F087FCF765FE8246A87A207405F10B0887
:1035F00004F10809002705E018F8010B09F8010B90
:10360000781CC7B2082FF7D36E68F08A18B13069FA
:103610000068206001E000202060F08AA080B08A6D
:10362000E0805046FCF748FE0020D8E710B50024A3
:103630000B480078012811D1FCF73AFE04460948EE
:10364000007840B908480078FF2804D2064800787E
:10365000401C054908702046FCF72EFE10BD0000F6
:103660002E000020210000202200002010B50024A0
:1036700013480078012821D1FCF71AFE04461148AE
:103680000078C0B91048007888B10F480078401E13
:103690000D4908700846007828B92046FCF70CFE52
:1036A00001F0F8F80AE02046FCF706FE06E02046A6
:1036B000FCF702FE02E02046FCF7FEFD10BD000014
:1036C0002E000020210000202200002070B50546B9
:1036D00000261048007808B1002070BDFCF7E8FD16
:1036E00006460D480468006820B10B480068406831
:1036F000094908603046FCF7DFFD4CB1032020701B
:1037000025810020606005A06061204600F008FF70
:103710002046E2E7210000200C0000203F000000CE
:103720002DE9F04105460E46144600272878032867
:1037300003D001202070BDE8F0813248007810B13C
:1037400002202070F7E73048007810B10D2020707B
:10375000F1E7FCF7ADFD0746288940B12889401EF6
:1037600028813846FCF7A8FD00202070E3E72748B1
:10377000006890F8340040F001002449096881F89D
:10378000340000202149096881F835001F4800688D
:103790000663284600F086FE3846FCF78DFD01F0F2
:1037A00079F8FCF785FD07461848006890F8350061
:1037B00020B1012809D0022806D102E000202070A3
:1037C0000BE00E20207008E000BF29460F4800687B
:1037D00000F034FE0A20207000BF00BF00200B491B
:1037E000096881F834000949096881F835000749FA
:1037F0000968C8610549096808623846FCF75CFD3C
:1038000000BF98E7210000202200002034000020A3
:1038100070B5044600252078032801D0012070BD32
:10382000FCF746FD0546A07A60B100230122194647
:10383000204600F0BBFD2846FCF73EFD01F02AF8CB
:103840000020ECE720894FF6FF71884207D22089DB
:10385000401C20812846FCF72FFD0020DFE728468A
:10386000FCF72AFD3320DAE710B50B48007890B951
:1038700001F04AF8094800780949087009480749E1
:10388000097850F82100084908600846006807498F
:103890000860FCF714FD10BD2E000020240000205D
:1038A00023000020180E00203C00002034000020DF
:1038B00010B50024022000F035FBFCF7F9FC0446AB
:1038C00000200B4908602046FCF7F6FC642000F05D
:1038D00029FBFCF7EDFC0446054800680549086033
:1038E0000120054908702046FCF7E6FC10BD0000E9
:1038F00030000020180000202000002010B50446F1
:103900002046FCF761FE10BD2DE9F04F85B08146E1
:103910008A4693461C46DDE90F78129D00200390ED
:10392000FCF7C6FC03902348007830B10398FCF7FD
:10393000C3FC3C2005B0BDE8F08F1F4850F82400C0
:1039400088BB01201C4941F824000398FCF7B4FC13
:103950002A464146384601F01BF92B465A46514645
:10396000484600F073F904901198CDE90080029563
:103970003A4620460E9B049900F0DCFF064636B915
:103980000E48007801280CD100F084FF09E0FCF714
:103990008FFC03900020084941F824000398FCF7AD
:1039A0008BFC3046C6E7FFE70398FCF785FC282030
:1039B000C0E7000021000020180E00202E0000208B
:1039C00010B504462046FCF700FE10BD2DE9F0417D
:1039D000054600274A48007810B14020BDE8F08134
:1039E0003F2D01D13E20F9E7FCF762FC0746FF2D91
:1039F00003D14448006890F83650434850F82540B9
:103A000024B93846FCF758FC4320E7E7012C04D1E1
:103A10003846FCF751FC3D20E0E714F8380F3B49ED
:103A2000085C617888432178384A505414F8380982
:103A30001146085C30B994F83A103548007888434C
:103A400033490870E06918B12046E16900F0F6FCDE
:103A5000206A18B12046216A00F007FDA66A16B157
:103A6000304600F097FD0020206384F8340084F88D
:103A7000350028480078FF2804D226480078401CEA
:103A8000244908703846FCF717FC00F08DFCFCF761
:103A90000FFC07461F48007820B11E480078401EE2
:103AA0001C490870204600F041F81B480078401E71
:103AB000194908700020144941F82500A06930B95F
:103AC00000206169886115496069086005E0D4E9F2
:103AD00005014861D4E905108861114800686061FA
:103AE0000F4804600FA020653846FCF7E5FB0E4840
:103AF0000078012801D100F0CDFE00206EE7000023
:103B00002100002034000020180E00202600002094
:103B100025000020220000202F000020400000206F
:103B2000380000203F0000002E00002010B50446A1
:103B30002046FCF74BFD10BD10B5FCF748FD10BD4D
:103B40002DE9F04106460F4614464FF0000815488F
:103B5000007818B112202070BDE8F081FCF7A8FBB6
:103B60008046FF2E03D11048006890F836600F4859
:103B700050F826502DB94046FCF79EFB432020709C
:103B8000EAE7012D05D14046FCF796FB4320207063
:103B9000E2E72F654046FCF78FFB0020207000BF56
:103BA000DAE700002100002034000020180E002079
:103BB00010B504462046FCF70BFD10BD10B5FCF710
:103BC00008FD10BD2DE9F04707460D464FF0000AED
:103BD000002028606860FCF76BFB8246FF2F03D152
:103BE0001848006890F83670174850F827402CB9EC
:103BF0005046FCF761FB4320BDE8F087012C04D15F
:103C00005046FCF759FB4320F6E7207C00F001000A
:103C100020B95046FCF750FB4520EDE70026D4F8CC
:103C20000C90D4F808805046FCF746FB00E0761C68
:103C300058F8041B0029FAD02E60A9EB0600686032
:103C40000020D9E734000020180E002070B504468B
:103C5000101D20F007004FF08076051F28462E60CB
:103C6000051F28462C60684E051F28462E604FF021
:103C70001236051F28462E604FF00336051F2846D2
:103C80002E604FF00236051F28462E607610051F65
:103C900028462E60051F284629604FF01136051F63
:103CA00028462E604FF01036051F28462E604FF034
:103CB0000936051F28462E604FF00836051F284696
:103CC0002E604FF00736051F28462E604FF006364F
:103CD000051F28462E604FF00536051F28462E602A
:103CE0004FF00436051F28462E6003F00405002D12
:103CF0007ED0F605051F28462E60444E051F284637
:103D00002E60434E051F28462E60424E051F284652
:103D10002E60414E051F28462E60404E051F284646
:103D20002E603F4E051F28462E603E4E051F28463A
:103D30002E603D4E051F28462E603C4E051F28462E
:103D40002E603B4E051F28462E603A4E051F284622
:103D50002E60394E051F28462E60384E051F284616
:103D60002E60374E051F28462E60364E051F28460A
:103D70002E604FF08346051F28462E60324E051FE9
:103D800028462E60314E051F28462E60304E051FF6
:103D900028462E602F4E051F28462E602E4E051FEA
:103DA00028462E602D4E051F28462E602C4E051FDE
:103DB00028462E604FF08246051F28462E60294E69
:103DC000051F28462E60284E051F28462E60274EC8
:103DD000051F28462E604FF08146051F28462E609D
:103DE000234E051F28462E603602051F284600E098
:103DF00009E02E604FF07E56051F28462E600026F3
:103E0000051F28462E6070BD9D4A00000000F84145
:103E10000000F0410000E8410000E0410000D8410E
:103E20000000D0410000C8410000C0410000B8417E
:103E30000000B0410000A8410000A04100009841EE
:103E40000000904100008841000070410000604186
:103E5000000050410000404100003041000020417E
:103E6000000010410000E0400000C0400000A04001
:103E7000000040402DE9F04105464FF00008FCF7F6
:103E800017FA8046FF2D05D12048006890F836507B
:103E9000012608E01D48006890F83600A84201D1CC
:103EA000012600E000261A4850F825402CB940466B
:103EB000FCF702FA4820BDE8F081012C04D140460D
:103EC000FCF7FAF94320F6E794F838701148C05D22
:103ED00094F8391088430F49C8550846C05D30B979
:103EE00094F83A100C48007888430B49087094F80D
:103EF000340040F0080084F834004046FCF7DCF958
:103F0000012E01D100F0C6FC0020D4E734000020CF
:103F1000180E0020260000202500002010B5FCF718
:103F200059FB10BD70B5054600261748007800B152
:103F300070BD1648007800B1FAE71DB3FCF7B8F978
:103F400006461348006890F838401248005D104952
:103F5000096891F8391088430E4908550846005DF4
:103F600040B90B48006890F83A100B480078884335
:103F7000094908700648006805633046FCF79CF95B
:103F800000F088FC00BFD3E72100002022000020C1
:103F900034000020260000202500002070B50025F8
:103FA000FCF786F90546034804682846FCF784F9BF
:103FB000204670BD5400002070B5002600F072F855
:103FC000FCF776F9064631480068401C2F49086026
:103FD0003046FCF771F92E480078012853D12D485E
:103FE000007820B1012804D0022809D103E001257E
:103FF0000BE0002509E0012501202649087004E0B6
:10400000012500202349087000BF00BF05B970BD1D
:104010002148046833E0FCF74BF90646206B50B3A7
:10402000206B401E2063206B28BB94F8340000F006
:10403000370040B114F8340F00F0C80020700120A0
:104040006070343C02E0002084F8350094F83400BD
:1040500000F0080078B93834A0781049097808438E
:104060000E49087020780E49085C6178084314F8FE
:1040700038190B4A505464693046FCF71DF994F81E
:1040800036003F28C7D100BFC1E700005400002020
:104090002E000020440000204000002025000020C9
:1040A0002600002010B5FCF796FA06480088401C50
:1040B000044908800846008818B10020088000F0F4
:1040C00003F810BD0400002010B503480068FFF796
:1040D0009FFB0446204610BD64000020F8B54FF455
:1040E0002071284800F078FB4021274800F074FB3D
:1040F000002514E0681C86B205EB8500214901EB20
:10410000C00406EB860001EBC0076420207000208D
:1041100084F82500E7601DA02062681C85B20F2D81
:10412000E8D305EB8500174901EBC004642020703B
:10413000002084F82500E06014A0206200201449CB
:104140000860144908801020134908800D4813495D
:1041500008600120FFF7BAFA114908600020FFF754
:10416000B5FA104908606A460FA10D480068FEF7CD
:10417000D1FF6A4611A10B480068FEF7CBFF00F0A3
:1041800027F8F8BDD8220020582700203F00000063
:104190005C0000205A000020580000206800002029
:1041A000600000206400002075432F4F532D4949C3
:1041B00020546D724C6F636B0000000075432F4FED
:1041C000532D494920546D725369676E616C00002C
:1041D00000B587B00320002180220A4BCDE90132CF
:1041E000CDE903104FF6FD703D23074A00900748C4
:1041F000FFF78AFB06AA06A13D20FFF7A1FC07B046
:1042000000BD000058250020542700208D420000EA
:1042100075432F4F532D494920546D720000000003
:1042200070B50B46032580F82550012B05D1154E9E
:10423000C5693668354445610CE085692DB9114E74
:10424000C56936683544456104E00E4E85693668B7
:1042500035444561057D05F007040B4D05EBC401B0
:104260000D682DB908600025C56001258D8006E028
:104270000A680860C26010618D886D1C8D80002501
:10428000056170BD5C0000205827002008B500BF04
:1042900000BF6A4600211A480068FFF741FAFFF79D
:1042A000C5F918480068401C16490860084600789F
:1042B00000F00708144800EBC8073C681AE0E668FD
:1042C000104960690968884213D1204600F01EF841
:1042D00094F82400022804D101212046FFF7A0FF12
:1042E00002E0022084F82500656815B12046A16827
:1042F000A8473446002CE2D1FFF7B8F9C9E700001F
:10430000640000205C0000205827002030B5057DA7
:1043100005F007040D4D05EBC4031D68854205D16A
:10432000C168196039B100250D6104E00169C268F6
:10433000CA6002B11161012580F825500025C560D1
:1043400005619D886D1E9D8030BD000058270020AE
:1043500010B5FBF7ADFF044606480078401C054940
:1043600008702046FBF7A8FFFFF726FEFEF752FF76
:1043700010BD00002100002001464A1E4FF0E0233E
:104380005A61084A106820F07F4000BF10601A464A
:10439000126942F005021A611A46126942F00202DD
:1043A0001A61704720ED00E0704700002DE9F04FE2
:1043B00005460F4690469946A87A1C490E5C05F1C1
:1043C0000B00805D11F800B00BEBC60000F0FF0A97
:1043D000174850F82A4000202434E0602760207CF1
:1043E00020EA0800207484F81190207C243C00F01E
:1043F000080068B994F83A000E49097808430D4955
:1044000008700D48805D94F8391008430A498855B2
:104410002946204600F012F8206A20B12046216A81
:1044200000F023F8E5615046BDE8F08F94B200003B
:10443000180E0020250000202600002010B590F85E
:10444000382001F10B039B5C90F83940A34301F144
:104450000B04A35423469B5C23B98B7A90F83A4013
:10446000A3438B720023C36110BDF0B5024612F85E
:10447000384F95785678383A0B4618680FE000F1B7
:104480000B073F5DB74300F10B0C0CF80470674657
:104490003F5D17B9877AAF4387721B1D18680028E4
:1044A000EDD1F0BD10B51B4A1268D061194A1268EF
:1044B00092F8383000F10B02D25C164B1B6893F86F
:1044C00039301A43134B1B6893F8384000F10B0343
:1044D0001A55827A0F4B1B6893F83A301A4382724E
:1044E0000C4A126892F838100B4A525C094B1B6850
:1044F00093F839309A43084B5A541A46525C42B9E1
:10450000044A126892F83A30044A12789A43034BEC
:104510001A7010BD34000020260000202500002065
:10452000014600228A72002005E0002301F10B02FF
:104530001354421CD0B20828F7D370472DE9F0413C
:10454000A021114800F048F900250DE0681C86B252
:104550000D4800EB051400EB061700202070676083
:104560000AA0E060681C85B2092DEFD3064800EB75
:10457000051400202070606004A0E0600248044937
:104580000860BDE8F0810000780900203F000000CD
:104590001000002030B501464A6808682AB9CC6886
:1045A000606028B10025456002E0106000B1426003
:1045B0008B6800259D6230BD70B54FF4BD61134816
:1045C00000F00AF9002411E0601C85B204EB4400FD
:1045D0000E4901EBC00305EB450001EBC0060020CE
:1045E00018705E600AA05861601C84B23E2CEBD348
:1045F00004EB4400054901EBC0030020187058602B
:1046000003A0586108460349086070BD900300206C
:104610003F0000000C00002000200B4908600B49FF
:1046200008700B4908700B4908700B4908700B495A
:1046300008600B4908600B4908600B4908600B498A
:1046400008700B49087070475400002021000020BA
:10465000220000202F0000202E0000200800002053
:10466000300000201C000020180000202000002046
:104670005000002000210A4A1170002004E00021AF
:10468000084A1154411CC8B20828F8D30021064A30
:104690001170064A1170064A1160064A116070478F
:1046A00025000020260000202300002024000020F8
:1046B0003C0000203400002070B54FF48F511948A1
:1046C00000F08AF84FF48071174800F085F8002454
:1046D00013E0601CC5B204EB440000EBC4001149B8
:1046E00001EBC00305EB450000EBC50001EBC00684
:1046F0005E610EA01865601CC4B2332CE9D304EBD4
:10470000440000EBC400074901EBC00300205861DE
:1047100006A018650020064908600248054908609F
:1047200070BD0000180F0020180E00203F00000090
:10473000400000203800002000B587B00320002191
:1047400080220A4BCDE90132CDE903104FF6FF700C
:104750003F23074A00900748FFF7D6F806AA06A1AC
:104760003F20FFF7EDF907B000BD0000180C002056
:10477000140E0020754A000075432F4F532D4949F0
:104780002049646C6500000000B587B0032000215B
:1047900080220A4BCDE90132CDE903104FF6FE70BD
:1047A0003E23074A00900748FFF7AEF806AA06A185
:1047B0003E20FFF7C5F907B000BD0000180A002031
:1047C000140C0020B54A000075432F4F532D494962
:1047D000205374617400000004E0002200F8012BF3
:1047E0004A1E91B20029F8D17047000070B5F0213F
:1047F0001148FFF7F1FF00240EE004EB44000E49DE
:1048000001EBC005601C00EB400001EBC0006860DC
:104810000AA06861601C84B2092CEED304EB44004A
:10482000054901EBC0050020686004A068610846E6
:104830000349086070BD0000F82000203F00000020
:10484000480000202DE9F041F0211048FFF7C4FF97
:1048500000240DE0601C86B204EB44000B4901EB20
:10486000C00506EB460001EBC0072F60601C84B258
:10487000092CEFD304EB4400044901EBC0050020F0
:104880002860084602490860BDE8F081E821002060
:104890004C00002010B50024FBF70AFD0446134825
:1048A0000078F8B912480078E0B900F02DF8114806
:1048B0001149097850F82100104908600E48007825
:1048C0000F49097888420DD00C480068C06B401C25
:1048D0000A490968C8630B480068401C0949086018
:1048E000FBF701FD2046FBF7E7FC10BD210000208F
:1048F00022000020180E0020240000203C00002090
:1049000023000020080000200649074A1278885C2E
:104910000649095C034A515C01EBC001044A11706D
:104920007047000094B200002500002026000020FF
:10493000240000202DE9F84F05460F469046994681
:10494000DDE90AAB00200090FBF7B2FC0090424882
:104950000468002C7BD01C3454F8080C3E490860D5
:104960000098FBF7A9FC44F81C7CA5760020207673
:104970006076606144F818BC44F810AC44F8148CBC
:104980000C9824F80C0C24F80A9C0020E077E8101E
:10499000207705F00700E076217F01208840A0778E
:1049A000E17E012088406077002020606060E06048
:1049B000A0602062A0626062E062206327A0606362
:1049C0001C3C002606E0002104F1540040F82610AB
:1049D000701CC6B2002EF6D02046FEF78FFFFBF704
:1049E00067FC00901E4840F825400098FBF764FCE7
:1049F0002046FEF7E5FFFBF75BFC009019480068D6
:104A000060610020A0611748006810B11548006877
:104A10008461144804603834A07813490978084345
:104A20001149087020781149085C6178084314F82E
:104A300038190E4A50540E480078401C0C49087032
:104A40000098FBF739FC0020BDE8F88FFFE70098DD
:104A5000FBF732FC4220F7E7380000203F0000005F
:104A6000180E002040000020250000202600002015
:104A70002F000020002400BF00BFFBF719FC0446F4
:104A800005480068401C044908602046FBF714FCF8
:104A9000FFF752F8F1E700003000002010B504489D
:104AA0000068FFF785F8FF20FEF790FF10BD0000BB
:104AB0003400002000BF00BF02E0C820FFF732FA38
:104AC0001F4800780028F8D01E4800686421B0FB19
:104AD000F1F01C4908600846006828B900201A490E
:104AE0000870FF20FFF7C6F9FBF7E2FB0446154804
:104AF000006864214843154908602046FBF7DCFB49
:104B000000BFFBF7D5FB0446104800681049086059
:104B100000200E4908602046FBF7CEFB0C480068D9
:104B200008490968B0FBF1F0C0F16400064908705B
:104B3000FFF744F800F00EF86420FFF7F3F9E0E720
:104B40002000002018000020140000203000002069
:104B50001C0000207CB5002514E069462846FFF7BC
:104B600031F8064666B9094850F8254044B1012C91
:104B700006D0D4E9020100EB8100A0640198E06452
:104B8000681CC5B23F2DE8D97CBD0000180E00207E
:104B900002F0010343B102F002032BB102E0491E0F
:104BA000002308C00029FAD17047000010B5002387
:104BB0001A460E490120FCF737FE0446002C02DAA3
:104BC0004FF0FF3010BD0120094988750948886100
:104BD0000948C8610846FCF7E8FC0446002C02DAE4
:104BE0004FF0FF30EEE70020ECE70000801A0600EF
:104BF000102E0020751C0000BD24000070B5044676
:104C00000D4616460CB9002070BD0DB90020FBE71B
:104C100021462A46002304E010780870491C521CE3
:104C20005B1C21B11AB1107808B1B342F4D301B1C1
:104C30000AB90020E8E7B34201D2002008702046FC
:104C4000E2E710B502460B461146002001E0491C80
:104C5000401C19B10C780CB19842F8D310BD00007B
:104C600010B50121C0F30722094B1A4402F070422B
:104C700042F00072C0F30723054C2344C3F313032F
:104C800042EA4312C3B242EA8302116010BD00003F
:104C900000E60F400146C1F307200B4A104400F024
:104CA000704040F00070C1F30722074B1A44C2F372
:104CB000130240EA4210CAB240EA8200006808B11A
:104CC000012070470020FCE700E30F400146C1F3DC
:104CD00007200B4A104400F0704040F00070C1F310
:104CE0000722074B1A44C2F3130240EA4210CAB229
:104CF00040EA8200006808B1012070470020FCE70C
:104D000000EA0F4018B50121C0F30722184B1A44DE
:104D100002F0704242F00072C0F30723144C2344A7
:104D2000C3F3130342EA4312C3B242EA830211609F
:104D30000021009102E00099491C0091009910297E
:104D4000F9D30021C0F30722094B1A4402F0704244
:104D500042F00072C0F30723054C2344C3F313034E
:104D600042EA4312C3B242EA8302116018BD000056
:104D700000E50F4001480068704700007400002003
:104D80002EE000241DE004EB4410164901EB400026
:104D90004078012813D104EB441011F81000401C96
:104DA00004EB44110F4A02F8110004EB44101146C1
:104DB00011F810003C2802DD01200B490870601C2E
:104DC000C4B2082CDFDB08480078012802D1FEF7C6
:104DD0008DF801E0FEF73AF84FF47A70FFF7A2F889
:104DE000CFE70000782F01207001002010B5FEF7FA
:104DF00033F810BD70477047816841F00101816050
:104E000070470121C16070470121C0F8001C704744
:104E100001607047816841F00201816070470000C5
:104E20000149C0F8001C704751E5CC1A7FB588B025
:104E3000DDE91045E0B28DF818004FF47F4104EA37
:104E400001000021000A40EA0160C0B28DF819009B
:104E50004FF47F0104EA01000021000C40EA014008
:104E6000C0B28DF81A004FF07F4104EA0100002122
:104E7000000E40EA0120C0B28DF81B00E8B28DF8A8
:104E80001C004FF47F402840000A8DF81D009DF85B
:104E9000200000069DF8211040EA01409DF82210F4
:104EA00040EA01209DF82310084305909DF8240056
:104EB00000069DF8251040EA01409DF8261040EAC2
:104EC00001209DF82710084304909DF82800000653
:104ED0009DF8291040EA01409DF82A1040EA01207F
:104EE0009DF82B1008430390FFF744FF064600216E
:104EF0000398CDE9000106A93046DDE9043201F04E
:104F00008BF80CB070BD000000BF0348806900F052
:104F100001000028F9D1704700F00A4002E008C8FB
:104F2000121F08C1002AFAD170477047002001E023
:104F300001C1121F002AFBD17047000010B50446C2
:104F400000F0BAFB0022034941F2883002F02CFB4A
:104F500010BD00003D4F00002DE9FC470546884686
:104F6000164600BF0DB9BDE8FC8700BF70892A282E
:104F70000EDA4B48408C401C81B249484184C08BBA
:104F8000401C81B24648C183304602F02BF8EAE764
:104F9000776807F10E042088B0F5807F08D120796A
:104FA000062805D16079042802D1608808280ED02F
:104FB0003B48008D401C81B239480185C08B401CA4
:104FC00081B23748C183304602F00CF8CBE7344851
:104FD000408B401C81B232484183D4F80E000190CE
:104FE000A0690090281D08B1686810B94FF0000949
:104FF00007E000986968884201D1012000E00020A4
:105000008146B9F1000F01D0012000E002200346E3
:1050100004F1080201A9284600F094FBE088B0F5ED
:10502000807F03D0B0F5007F2DD12BE0B9F1000FC8
:1050300026D0022001F0ADF8E080D4F80E00A06187
:105040006868C4F80E0000BF00BFA068C4F8120072
:10505000A089E082A0683860A089B880D8F80000F4
:10506000A060B8F80400A081D8F80000C7F80600D6
:10507000B8F80400788131462846AA69904700E0D4
:1050800000BF07E006E00648808D401C81B204485E
:10509000818500BF00BF304601F0A4FF00BF62E77A
:1050A000040201202DE9FC5F05460F464FF00A0877
:1050B000C1460A260024A34600200190B246009073
:1050C00000BF5CE004EB84004D4A02EB8000817C71
:1050D0000A2E02D109B966B24FE000294DD000BFB7
:1050E00000BF5DB104EB8402454B03EB82022868EC
:1050F0005268904202D160B2BDE8FC9F012928D1DC
:1051000004EB84003E4A52F8200088B104EB84008E
:1051100002EB8000C27C009882422EDB4FFA84FAB8
:1051200004EB8400364A02EB8000C07C009024E04F
:1051300004EB8400324A02EB8000C07C58451CDB43
:105140004FFA84F804EB840002EB800090F813B06F
:1051500013E0022911DB04EB8400294A02EB8000F2
:10516000C27C0198824208DB4FFA84F904EB840088
:10517000234A02EB8000C07C0190601CC4B20A2C60
:10518000A0DB07F0020020B90A2E05D107F00100CC
:1051900010B94FF0FF30AFE70A2E01DAF4B21AE08F
:1051A000B9F10A0F03DA09F0FF0400BF0EE0B8F10D
:1051B0000A0F02DA08F0FF0408E0BAF10A0F02DA77
:1051C0000AF0FF0402E04FF0FF3095E700BF00BF98
:1051D000204600F017F800BF00BF00BF00BF35B188
:1051E00004EB8401064A02EB810128684860002034
:1051F00004EB8401024A02EB8101C87460B27BE7D0
:105200003803012010B5044604EB84000C4951F822
:10521000200060B104EB8401094A52F8210001F03A
:10522000E1FE002004EB8401054A42F82100002041
:1052300004EB8401024A02EB8101887410BD000076
:10524000380301202DE9FC4704460F461546A946C0
:1052500000BF00BF00BF00BF00BF00BF0E21384627
:1052600001F025FF40B14B484089401C4949488125
:105270006FF00100BDE8FC872146286800F0A3FC20
:1052800010B1DFF814817DE0287800F0F000E0280C
:1052900015D101208DF8000000208DF801005E205E
:1052A0008DF80200687800F07F008DF80300A87880
:1052B0008DF80400E8788DF80500E84661E028687C
:1052C000A1680840D4E901121140884210D0288812
:1052D00080B24FF6A96188420AD004F10C0020B1D7
:1052E000E06810B104F10C0902E06FF00300C1E7BF
:1052F0002A48007800EB8000294901EB8000807C7F
:10530000022818DB2549097801EB8101244A02EBC8
:105310008101D9F80000496888420CD11D48C08D30
:10532000401C81B21B48C1851C4802783946204682
:1053300000F038F89EE700261BE006EB86001849CF
:1053400001EB8000807C022811DB06EB8601144A09
:1053500002EB8101D9F800004968884207D10F4962
:105360000E70F2B23946204600F01CF882E7701C3D
:1053700046B20A2EE1DB3A464946204600F048F89C
:1053800078E700BF434604F12F023946204600F07B
:1053900077F96FE70402012014B500001201002024
:1053A0003803012070B505460E46144600BF00BF05
:1053B00004EB8400154901EB8000807C022817D1A2
:1053C00004EB840001EB8000C07CE42810DB04EBDC
:1053D00084000A4602EB8000011D284600F03AF9DD
:1053E00030B9032004EB8401084A02EB8101887480
:1053F00004EB8400054901EB800000F10C0305F18A
:105400002F023146284600F03BF970BD38030120D9
:105410002DE9F05F80460F46164608F12F094FF040
:10542000FF3A4146386800F0CEFB38B9387800F0D2
:10543000F000E02802D00FB1386818B96FF00D0005
:10544000BDE8F09F01213846FFF72CFE0446002CF2
:1054500008DA2EB14948808C401C81B247488184CB
:105460002046EDE704EB8400454901EB8000807C99
:1054700030B9012004EB8401414A02EB81018874B8
:1054800000BF00BF04EB84003D4901EB8000807C3D
:10549000012800D03EB93946404600F0DBF882468C
:1054A0000EB95046CCE700BF00BF04EB840034497E
:1054B00001EB8000807C02280FDB32490C7004EB8A
:1054C00084002F4901EB800000F10C034A4631466D
:1054D000404600F0D5F882464EE004EB84002849AF
:1054E00001EB8000807C012846D14FF0000B35464F
:1054F00008E000BF00BF287B012802D04FF0010B5D
:1055000002E02D68002DF4D100BFBBF1000F10D0D8
:1055100029890022032001F0A7FB05466DB1314621
:10552000284601F0B6FC40B1284601F05BFD00259D
:1055300003E03546284601F059FEA5B104EB84008E
:105540000F4951F8200030B104EB84010C4A52F8A5
:10555000210001F047FD04EB8400094941F8205087
:105560004FF0000A07E00548808C401C81B20348D8
:1055700081844FF0FF3A00BF504661E704020120EA
:1055800038030120120100202DE9F84F0746884614
:1055900091469A46DDF828B00020009000BF00BF79
:1055A00000222A21032001F05FFB05464DB928485F
:1055B000808C401C81B2264881844FF0FF30BDE8CA
:1055C000F88F00BF00BF6E6806F10E040D9800F062
:1055D000E0FDE08000BF00BFDAF80000A060BAF88C
:1055E0000400A0810B980168C4F812108088E08242
:1055F000D9F800003060B9F80400B080D8F8000095
:10560000C6F80600B8F804007081DBF80000C4F8A2
:105610000E000C980068A0614FF480702080082074
:10562000608006202071042060714FF4C160B08159
:1056300029463846BA69904700900548008B401CBF
:1056400003490883284601F0CDFC00250098B6E701
:10565000040201207FB504460D460121064A201DA3
:1056600004F12F038DE825000391044A19462046D2
:10567000FFF78AFF04B070BD1AB5000014B5000032
:105680002DE9F04105460E4617469846746800BF5E
:1056900000BFD8F800002060B8F80400A080386887
:1056A000C4F80600B88860810820A08131462846E9
:1056B000AA699047BDE8F08170B500243DE004EB95
:1056C00084001F4901EB8000857C25B304EB840036
:1056D00001EB8000C07C401C04EB8401184A02EB03
:1056E0008101C87404EB8400114601EB8000C07C8A
:1056F000F0280DDA04EB840001EB8000807C0128A7
:105700000AD104EB840001EB8000C07C022803DB9B
:105710002046FFF777FD0EE004EB8400084901EB1B
:105720008000807C032806D1022004EB8401044A17
:1057300002EB81018874601CC4B20A2CBFDB70BD0F
:10574000380301202DE9F04706460D4617469846D6
:1057500000BF00BF5DB1286848B13146286800F03D
:1057600032FA20B9287800F0F000E02803D16FF079
:105770000D00BDE8F08741462846FFF793FC04463C
:10578000002C01DA2046F4E7022004EB84011A4AD7
:1057900002EB8101887404EB8400114601EB800068
:1057A000866004EB840001EB80003968C160B98831
:1057B0000182002004EB840102EB8101C87404EB38
:1057C0008400114651F8200098B104EB840051F890
:1057D0002090002004EB840142F821003B4606F1B2
:1057E0002F0249463046FFF74BFF484601F0FAFBCF
:1057F00000BF0020BDE70000380301202DE9F04183
:1058000004460E464FF00E0860890E280BDC334824
:10581000008D401C81B231480185C08B401C81B293
:105820002E48C18354E06568AF89287800F00100F4
:10583000B0B12878012809D1687888B9A8785E289D
:105840000ED1607B40F01000607309E0062224490D
:105850002846FAF7DDFD18B9607B40F00800607358
:10586000082F03D0B7F5C16F22D114E096F83500A8
:1058700000F0200000B92BE0C8F1000001B2204682
:1058800001F015FC10B100BF00BF21E031462046F9
:1058900000F0C0F918E096F8350000F0200000B9DB
:1058A00016E0224606F12F013046FFF755FB0BE0CC
:1058B0000A48008D401C81B208480185C08B401CFD
:1058C00081B20648C18303E000BF0020BDE8F0813B
:1058D000204601F087FB0020F8E7000004020120C9
:1058E00014B5000070B505460C4622460321284633
:1058F00000F0F2F870BD00002DE9FE4F0446894625
:105900007248B0F84A00401C81B27048A0F84A10B2
:105910006568287800074FEA9068C8F100012046C2
:1059200001F0C5FB10B92089042800D2B4E06068FA
:1059300090F800A0BAF1000F03D0BAF1080F7DD1A2
:1059400000E0A4E001266248007800F0F000E028C2
:1059500000D100265E490868494600F034F900B1DC
:10596000002666B95948B0F85C00401C81B257481F
:10597000A0F85C10204601F035FBBDE8FE8F2089C1
:10598000082800D288E0204600F0F2F858B12046FE
:1059900001F028FB4D48B0F85000401C81B24B4844
:1059A000A0F85010E9E72421204601F080FB48B31D
:1059B0004146204601F07BFB10B100BF00BF77E0FD
:1059C00021890022022001F04FF9064606B96FE056
:1059D00000BF00BF2146304601F05BFA10B100BFA6
:1059E00000BF65E07568C8F1000001B2304601F003
:1059F0005EFB10B100BF00BF5AE0204601F0F2FA92
:105A0000344608E06FF02301204601F050FB10B14E
:105A100000BF00BF4CE067682D480068E8602D4873
:105A200000682861002038707880FF2028720020EC
:105A300068812648B0F84800401C00E017E0234980
:105A4000A1F848004146204601F031FB08B100BFF3
:105A50000CE001200021FF230A46CDE90109009155
:105A60001B49204600F0FEF9064600BF0FE017482C
:105A7000B0F85800401C81B21448A0F85810B0F893
:105A80004E00401C81B21148A0F84E1000BF00BF6C
:105A9000204601F0A7FA70E7204601F0A3FA0B4870
:105AA000B0F85200401C81B20848A0F8521064E7D8
:105AB000204601F097FA0548B0F85C00401C81B21E
:105AC0000248A0F85C1000BF57E700000402012064
:105AD0000C010020080100202DE9FE4306460F4678
:105AE000904600222421012001F0BEF805460DB9A0
:105AF000BDE8FE8300BF00BFD6F804906C68277035
:105B000084F801800020A080E08071686A6802F15A
:105B100008001C22FAF73EFC0020608069892046BC
:105B200000F01CF860800C48B0F84800401C0A499E
:105B3000A1F84800D9F80C00029001200021FF23B1
:105B400002AACDE90010284600F068F9284601F0C5
:105B500049FA00BFCCE700000402012070B50446FA
:105B60000D462946204600F03BFBC04380B270BD85
:105B70002DE9F041064600240027354617E06989E3
:105B8000686800F02DFB0444A0B200EB144468895F
:105B900000EBD0714910A0EB410139B1C7F1010010
:105BA000C7B2E0B2C4F3072141EA00242D68002DFA
:105BB000E5D127B1E0B2C4F3072141EA0024E04374
:105BC00080B2BDE8F08118B502460092D04300B122
:105BD0000AB9012018BD91F8350000F0020008B99B
:105BE0000020F7E74868904201D10020F2E70098D2
:105BF0008B681840D1E901342340984208D1886865
:105C000022EA00008C68E343984201D10120E1E7D9
:105C10000020DFE72DE9F04706460F467948408E21
:105C2000401C81B277484186756828780421B1EB21
:105C3000201F12D0304601F0D5F97248B0F8440068
:105C4000401C81B26F48A0F84410C08E401C81B245
:105C50006C48C1860020BDE8F087287800F00F0965
:105C60004FF6FF7000EA8909688800F0B2FA8046B2
:105C70007089484502DB308940450FDA304601F033
:105C8000B1F96048408F401C81B25E484187C08EA8
:105C9000401C81B25B48C1860020DCE741463046AB
:105CA00001F068FA286958490860E86857490860AF
:105CB0004FF0010A3C4600BF94F8350000F00100A7
:105CC00078B1201D68B1606858B14F4800686168BC
:105CD000884205D04C4908682146FFF774FF00B19F
:105CE0000DE0BAF1000F04D04FF0000A48480468F4
:105CF00000E02468BC4200D12468002CDCD100BF45
:105D0000424908683946FFF75EFF28B93F480078E6
:105D100000F0F000E0280AD1304601F063F939487C
:105D2000C08E401C81B23748C186002093E724B959
:105D3000304601F057F900208DE7E8884FF63F71B3
:105D4000084088B1304601F04DF92E48B0F84200C5
:105D5000401C81B22B48A0F84210C08E401C81B27A
:105D60002848C186002076E72A4807602A4805604F
:105D70003946304601F08CFAC0BB687A01280DD054
:105D8000062806D011280ED13946304604F09EFF71
:105D90002BE03946304602F055F826E039463046C9
:105DA000FFF7AAFD21E0184908683946FFF70BFF05
:105DB00050B91548007800F0F000E02804D0756074
:105DC00002213046FFF78EFD304601F00BF90D48F9
:105DD000B0F84000401C81B20A48A0F84010C08EC4
:105DE000401C81B20748C18600BF00BF002009499E
:105DF000086009490860054908600349086000BF58
:105E000029E70000040201200C0100200801002005
:105E10009C00002000010020040100202DE9FE4F1D
:105E200006460F4615469846DDE90C9A00BF00BFAE
:105E3000284600F07DF8041E08D10948C08F401C98
:105E400081B20748C187201FBDE8FE8F43462A461E
:105E500039463046CDE9009A029400F003F8F3E7A2
:105E6000040201202DE9F84F05460E4617469A46D2
:105E7000DDF828B0DDF8308000BF00BF002F43D030
:105E80004FF014091421284601F011F958B12648A1
:105E9000B0F84400401C81B22348A0F844106FF0D1
:105EA0000100BDE8F88F6C6800BF00BF84F808A04F
:105EB0000B9860723868206148464FEAE97109EB37
:105EC0009171C1F3870141F04001217084F801B064
:105ED000288900F05EF960800020E0801348008887
:105EE00000F057F9A08011480088401C0F49088035
:105EF0000EB1306818B9D8F80400E06001E03068ED
:105F0000E0600020608103E06C68206900906F46CB
:105F10000548008E401C044908863A4629464046FA
:105F2000D8F814309847BCE7040201201001002083
:105F300010B50246144801680FE091F8350000F0F2
:105F4000010048B110688B681840D1E90134234042
:105F5000984201D1084610BD09680029EDD10B48CF
:105F6000006830B10948006890F8350000F0010081
:105F700038B90748C08F401C83B20548C38700204A
:105F8000E9E702480068E6E79C000020A000002046
:105F90000402012070B50025FDF722F9FAF788F90F
:105FA000054601211848FBF7A7F8044604F0805085
:105FB00050B11548FBF74DF91348FBF734F9124877
:105FC000FBF71BF924F080541CB121460E48FBF767
:105FD00055F804F0005058B10B48FBF72FF906466E
:105FE0000A48006820B131460748084A12689047BD
:105FF0001CB12146064804F0D5FB2846FAF75CF9A7
:10600000FDF708F970BD000000C00E405C010020E3
:106010003C2F0120704700002DE9FC4704460D4647
:1060200016461F46DDE90A892248FEF719FE214877
:10603000FEF768FE2048FEF72DFE30B11E48FEF741
:106040000FFE1D48FEF75EFE01E000BFFEE700BF49
:106050001848FEF73BFE0028FAD040F20E411748E0
:10606000FBF764F8002004210B46154ACDE9001027
:1060700021461248FAF7AEFF00234FF008724FF4A2
:1060800040610E48FAF784FF2A4600210B48FAF7D0
:1060900042FF0C48C0F800900B4806600B480760B0
:1060A0000B48C0F8008000210A4804F0A7F9BDE8B9
:1060B000FC870000009C00F0003000F000C00E40A3
:1060C000020000046001002064010020680100203B
:1060D0006C010020F160000010B50446FFF79AFF44
:1060E00000220249012001F05FFA10BDD9600000D2
:1060F00010B586B004461848006878B9174800689B
:1061000000F03AF805901648006800F035F8049061
:106110001448006800F030F8039003E00020059078
:106120000490039010481149002203ABCDE90021EF
:10613000029004AA05A90E4800F0A0FC0C4800F04B
:10614000EBFC0B4800F06DFD00220A49012001F034
:106150002BFA06B010BD0000600100206401002091
:10616000680100206C01002061A4000065A7000008
:106170003C2F0120D96000000146080601F47F424F
:1061800040EA022001F47F0240EA122040EA116056
:10619000704701460806000C40EA1120704710B510
:1061A00001F0B0F801F032F900F0CEF800F0B2FAE8
:1061B00000F09CFC00F013F804F086FD01F040FEB6
:1061C00001F05CFA10BD00B503461846FFF7D4FF96
:1061D00000BD00B502461046FFF7DBFF00BD70476B
:1061E000F8B505460A462B4600200090002103F032
:1061F000010636B1002A04DD13F8010B8DF8010009
:10620000521E1C4603E034F8027B3944921E012AD8
:10621000F9DC002A02DD20788DF80000BDF80000CE
:10622000014488B200EB114188B200EB114126B164
:10623000C8B2C1F3072747EA002188B2F8BD0000C1
:1062400088B006A90FA0FAF7D3FDFAF789F8FCF792
:106250008DFF032000214FF400720E4BCDE9013277
:10626000CDE90310022003460B4A00900B48FDF7CE
:106270004BFB07AA0AA10220FDF762FCFDF7F4FA26
:1062800000BFFEE7544D3443313239584E435A4132
:106290004400000008320120043A012035050000C6
:1062A000537461727400000070B5054605B970BD85
:1062B00000BF00BF00BF00BF1E480068854203D377
:1062C0001D48006885420FD3002601F063F806469A
:1062D0001A48B0F89800401C81B21848A0F89810ED
:1062E000304601F08DF8E2E70021154801F056F83C
:1062F000A5F1080400BF00BF00202071114800680C
:10630000844201D20F48046020880A490988611A32
:10631000411A0A48B0F89200401A81B20748A0F822
:106320009210204600F070FF054801F0FDF800BF14
:10633000BDE700008C000020900000200402012036
:10634000980000209400002010B500BF00BF17483F
:1063500020F0030016490860084604684FF42050F6
:1063600020800020608020710846006800F52050E1
:10637000104908600120096808714FF420500D4948
:10638000096808800B4909684880094800680A497B
:1063900008604FF420500949A1F8900001210848F5
:1063A00001F0A8F808B100BF00BF10BD332E0020D7
:1063B0008C000020900000209400002004020120A6
:1063C000980000202DE9F041054615B90020BDE8F0
:1063D000F081E81C20F0030085B20C2D00DA0C25BA
:1063E000B5F5205F01DD0020F1E70021524800F003
:1063F000D5FF5248008852490988401A86B289E080
:106400004F4800688419207900287CD1218806F142
:106410000800081AA8427AD3218806F10800091A50
:1064200005F11400814232D306F1080028441FFA16
:1064300080F84348006800EB080700203871208886
:1064400038807E80A4F80080012020713888B0F563
:10645000205F05D038883A4909680844A0F80280CE
:1064600000BF3848B0F8921005F10800084481B226
:106470003448A0F89210B0F89410B0F8920081421D
:1064800004DA3048B0F89210A0F894101BE0012014
:10649000207100BF20882A490988611A411A2948B9
:1064A000B0F89200084481B22648A0F89210B0F8E3
:1064B0009410B0F89200814204DA2248B0F89210A9
:1064C000A0F8941000BF1D480068844211D11B49F8
:1064D000086803E001881A4A12688818017919B11E
:1064E000194909688842F5D11449086000BF00BF06
:1064F00000BF114801F018F800BF00BF00BF00BF87
:1065000000BF00BF00E002E004F108005FE70C48B4
:106510000068865BC5F52050B0423FF771AF09486F
:10652000B0F89600401C81B20648A0F896100248C8
:1065300000F0FAFF00204AE79800002094000020B5
:106540008C00002004020120900000202DE9F05F63
:1065500082460D46E81C20F0030085B20C2D00DABF
:106560000C25B5F5205F02DD0020BDE8F09F00BFDF
:1065700000BF4B480068824503D34A480068824503
:1065800011D34FF0000B00F005FF83464648B0F8EA
:106590009800401C81B24448A0F89810584600F07A
:1065A0002FFF5046E1E7AAF108073D480088381A56
:1065B0001FFA80F93888A0EB090008381FFA80F824
:1065C00000BF00BF454501DD0020CEE7454501D1B4
:1065D0005046CAE70021354800F0E0FE38883049CF
:1065E00009684418207950BB208809F10801294422
:1065F0008EB22F490968A14204D129490968314462
:106600002B4A1160264909688C19002121712080CC
:10661000A4F802903E802188B1F5205F04D0218843
:106620001F4A126811444E801F49B1F89210A8EB1E
:106630000502891A8AB21C49A1F892202AE005F1C4
:106640001400404526D809F10800284486B21448B1
:106650000068841916480068844201D21448046016
:106660000020207138882080A4F802903E80208885
:10667000B0F5205F04D020880949096808444680A5
:106680000948B0F89200A8EB0501401A81B206480B
:10669000A0F89210054800F047FF504665E700005B
:1066A0008C000020900000200402012098000020AF
:1066B000940000202DE9F04104460D4600270DB955
:1066C000BDE8F08100BF00BFA5F11C0600F062FE2E
:1066D000074600F0DBF804EB84010C4800EB4100B6
:1066E0004088401E81B204EB8402084800EB42005F
:1066F0004180074850F824003060054840F8246085
:10670000384600F07DFE00BFDAE700009E0201205F
:106710004456002070B500241CE0002104EB8402E4
:10672000224800EB4200418004EB84021F4800EB4A
:106730004200818004EB84021C4800EB4200C180CF
:106740001B4830F8141004EB8402184820F812108B
:10675000601C84B20C2CE0DB164820F003050024FA
:106760001DE00020144941F82400002610E01248E2
:1067700050F824002860104840F824500F4830F8A2
:10678000141005F11C00084400F11005701C86B2BD
:10679000074830F81400B042E9DC601C84B20C2CCD
:1067A000DFDB00F033F900F071F870BD9E020120CC
:1067B000ACB30000775600204456002094B300008C
:1067C0002DE9F04104460E4617464FF0000800BF81
:1067D0000C2C02DB0020BDE8F08100BF00F0DAFDE8
:1067E000804600F053F8274850F82450ADB32549AF
:1067F000286841F82400002028606E60AF6000BF68
:1068000004EB8401204800EB41004088401C81B229
:1068100004EB84021C4800EB4200418004EB84013D
:10682000194800EB4100818804EB8402164800EB14
:106830004200408881420BDA04EB8401124800EBED
:106840004100418804EB84020F4800EB4200818044
:1068500000BF00BF00BF1C350EE0FFE704EB840162
:10686000094800EB4100C088401C81B204EB84025F
:10687000054800EB4200C180404600F0C1FD2846BB
:10688000A9E70000445600209E02012070B51F4871
:1068900020F00305002417E000BF00260DE021468C
:1068A000284600F039F81A4830F8141005F11C0099
:1068B000084400F11005701C86B2164830F8140028
:1068C000B042ECDC601C84B20C2CE5DB0F4820F0FD
:1068D0000305002417E000BF00260DE021462846EE
:1068E00000F05AF80A4830F8141005F11C0008446A
:1068F00000F11005701C86B2064830F81400B04252
:10690000ECDC601C84B20C2CE5DB70BD77560020FB
:1069100094B30000ACB30000F0B5A1B006460C463D
:106920001A4830F8141006F11C000F18002529E051
:10693000785DCD2824D08022154901A8F9F72AFDD9
:1069400014A0006800900A2C0ADB0A2094FBF0F0E7
:106950003030C0B28DF80000694601A8F9F73EFD5D
:106960000A2094FBF0F100FB11403030C0B28DF8EA
:106970000000694601A8F9F731FD00BF00BF00BF64
:10698000681C85B2102DD3DB21B0F0BD94B300009C
:10699000C4B3000030000000F0B5A1B006460C46BC
:1069A00006F10C07002529E0785DCD2824D080224F
:1069B000144901A8F9F7EEFC13A0006800900A2C16
:1069C0000ADB0A2094FBF0F03030C0B28DF80000F2
:1069D000694601A8F9F702FD0A2094FBF0F100FBDB
:1069E00011403030C0B28DF80000694601A8F9F7B7
:1069F000F5FC00BF00BF00BF681C85B2102DD3DBC3
:106A000021B0F0BD44B40000300000002DE9F04199
:106A1000174820F00305002425E000BF00261BE0F6
:106A200005F10C07CD2210213846F9F7C5FC1148B5
:106A300030F8141005F11C000F18CD221021384633
:106A4000F9F7BAFC0B4830F8141005F11C000844A3
:106A500000F11005701C86B2074830F81400B042EF
:106A6000DEDC601C84B20C2CD7DBBDE8F0810000BA
:106A70007756002094B30000ACB300002DE9F04736
:106A800004460D4616461F46DDE909A9DDF82080BB
:106A900000BF00BF00206060A060E06084F83500A7
:106AA000E0612062C4F828800E48007884F838003D
:106AB0000C480078401C0B490870C4F810903B4605
:106AC00032462946204600F012F82046D04710B141
:106AD0000020BDE8F0870448006820600248046098
:106AE0002046F6E7A40000209C00002070472DE916
:106AF000F04106460F4614461D463946304600F022
:106B000017F82146304600F086F82946304600F056
:106B100009F8BDE8F08100000149086070470000F5
:106B2000A000002009B9002200E00A68C260704796
:106B30002DE9F04107460C4654B320687968884235
:106B400001D1012000E0002010BB154806680BE0D1
:106B500030687968884206D1D6F80C80304600F05B
:106B600065FE464600E0F668002EF1D10D48056846
:106B70000CE055B1286840B128687968884204D192
:106B80000CB9002000E020682860ED68002DF0D1ED
:106B90000CB9002000E020687860BDE8F0810000BA
:106BA000BC000020B800002010B5044694F8350061
:106BB00000F0100060B194F8350020F0100084F867
:106BC000350000BF206A10B12046216A884700BF07
:106BD00010BD10B5044694F8350000F01000C8B997
:106BE00014F8350F40F01000207014F8350900F04B
:106BF000010040B194F8350000F0200018B1211DCB
:106C00002046FEF727FD00BF206A10B12046216A0A
:106C1000884700BF10BD09B9002200E00A68826001
:106C2000704710B5044694F8350000F00100D0B963
:106C300094F8350040F0010084F8350000BFE069A9
:106C400010B12046E169884700BF94F8350000F094
:106C5000100040B194F8350000F0200018B1211D5B
:106C60002046FEF7F7FC10BD2DE9F05F83460F4686
:106C70009046BBF1000F09D0BBF1010F08D0BBF16A
:106C8000020F07D0BBF1030F08D105E038260AE058
:106C9000242608E0102606E0002604E000BF00BF1E
:106CA0000020BDE8F09F00BFB8F1000F78D0B8F128
:106CB000010F72D0B8F1020F70D0B8F1030F6ED18E
:106CC000EF2256A10B20FFF77BFD04461CB900F014
:106CD0002DFA0020E5E784F80C800020206006F102
:106CE00010002044C01C20F00300606000BF00BF03
:106CF0002781F01C20F0030040F2EC51081AB84242
:106D000001DD384605E0F01C20F0030040F2EC51B4
:106D1000081A608100BF00BF00BF00BF0120E081F2
:106D2000A2466089A7EB000932E04FF488723BA1CC
:106D30000B20FFF745FD054635B900F0F7F9204671
:106D400000F050F90020ACE785F80C800020687353
:106D50002860CAF8005000BF00BFA5F808901FFACD
:106D600089F040F2EC51884202DA1FFA89F001E022
:106D700040F2EC50688105F11000686000BF00BF70
:106D800000BF00BF0120E8816889A9EB0009AA467D
:106D9000B9F1000FC9DC39E002E020E020E031E089
:106DA00006F1130121F00302F91C21F00301114443
:106DB00088B2FFF707FB04460CB9002071E704F125
:106DC00010003044C01C20F0030060602781678100
:106DD0000020206084F80C8000BF00BF16E000BFD8
:106DE0004FF4A3720DA10A20FFF7EAFC04460CB988
:106DF000002056E70020606027816781206084F8CA
:106E00000C8003E000BF00BF00204AE700BF012064
:106E1000E08100206073204643E700002E2E5C5383
:106E200072635C5573725C4472697665725C55700E
:106E30004472697665725C6C7769705C636F7265C9
:106E40005C706275662E630010B5024600BF02B129
:106E500001B910BD00BF104604E003890C8923442A
:106E6000038100680368002BF7D100BF00BF00BF9B
:106E700000BF03890C8923440381016000BFE8E758
:106E80000146002002E0421CD0B209680029FAD174
:106E900070472DE9F04105460C460026002700BF4B
:106EA00025B11CB128892189884203DA6FF00D00D1
:106EB000BDE8F08100BF00BF6889801B6189C91BE4
:106EC000884204DB6089C01B1FFA80F803E06889F0
:106ED000801B1FFA80F86268D1196A6890194246CF
:106EE000F9F758FA06EB080086B207EB080087B2FC
:106EF00000BF00BF00BF00BF6089B84201DC0027AF
:106F000024686889B04208D100262D6800BF1DB9E9
:106F100014B16FF00D00CBE700BF54B16089218937
:106F2000884206D100BF206810B16FF00500BFE7AE
:106F300000BF55B168892989884206D100BF2868F9
:106F400010B16FF00500B3E700BF002CB4D10020F2
:106F5000AEE72DE9F05F8046894616461D464FF0A4
:106F6000000B00BFB8F1000F02D10020BDE8F09F78
:106F700000BF00BFB9F1000F01D10020F6E700BF4C
:106F80004FF0000AB8F1000F02D0B9F1000F01D1A3
:106F90000020EBE7444620E035B16089A84203DCDD
:106FA0006089281A85B217E06089401B87B2B74212
:106FB00000DD37466268511909EB0A003A46F9F7D5
:106FC000E9F90BEB07001FFA80FB0AEB07001FFA39
:106FD00080FAF01B86B2002524680EB1002CDBD1AC
:106FE0005846C3E72DE9F047044624B900BF00BF67
:106FF0000020BDE8F08700BF00BF00262DE04FF065
:10700000000900F0C7F9814600BF00BFE089401EBB
:107010001FFA80F8A4F80E80484600F0F1F9B8F1A4
:10702000000F18D12768257B032D04D121460B20A2
:10703000FFF740FB0BE0012D01D0022D04D12146CA
:107040000A20FFF737FB02E02046FFF72DF9701CFE
:10705000C6B23C4600E0002400BF002CCFD1304631
:10706000C7E7000070B5002500F094F90546002040
:107070000A490870284600F0C3F90948046808E086
:10708000606F28B1606F02F068FE0020606770BD1D
:10709000E468002CF4D100BFF9E70000A50000204F
:1070A000BC00002010B50446FFF7DCFF10BD70B532
:1070B000024600BF00BF01B10AB9002070BD00291F
:1070C00008DA484284B200BF5089A04201DA0120A8
:1070D000F4E700E08CB2137B55680BB1032B0AD1A7
:1070E0005068401A506002F110005668864215D26E
:1070F00055600120E2E7022B01D0012B0AD10029C3
:1071000006DA5089A04203DB5068401A506005E05F
:107110000120D3E700BF00BF0120CFE7508908441A
:1071200050811089084410810020C7E770B5002500
:1071300000F030F905460D48047801200B4908702D
:10714000284600F05DF984B900BF002211460848C6
:1071500003F00CF940B100F01DF905460020034989
:107160000870284600F04CF900BF70BDA500002053
:10717000A57000002DE9F04106460F4600BF00BF94
:1071800000BF00BF3089B84201DCBDE8F081308922
:10719000A7EB00083D4634460AE06089281A85B20C
:1071A00000BF00BF208940442081246800BF00BF89
:1071B0006089A842F1DB207B60B96089A84209D0D0
:1071C000A088001B284481B22046FFF7BFF904467F
:1071D00000BF00BF658160892081206810B12068F0
:1071E000FFF700FF0020206000BFCEE770B5044627
:1071F000002544B100F0CEF80546E089401CE0814E
:10720000284600F0FDF870BD30B500BF00BF00BFDC
:1072100000BF00BF00BF00BF00BF0388194C246837
:107220001919884215D00B799BB9174B1B689942E5
:107230000FD0164B1B688B4201D1144B18600B8882
:107240000380104B1B88C31A0C880E4D2D682C44EC
:10725000638043880B4C24681A19824211D0137939
:107260007BB90A4B1B68834201D1084B1A60038823
:107270001380044B1B88D31A0488024D2D682C44BC
:10728000638030BD8C00002090000020940000201E
:107290002DE9F04705468A460027D5F8048098F87E
:1072A00009900026144804681FE0207C48451AD144
:1072B00034B1206820B1114920680968884212D190
:1072C000606980B10E4B2A462146D4E905C0E047EB
:1072D00048B10025012736B1E068F0600648006833
:1072E000E060054804602646E4680FB9002CDCD154
:1072F0003846BDE8F0870000A80000200C010020FF
:1073000008010020704700002DE9F84F81460E4625
:107310001446D9F800A04CB14FF47A7060434FF492
:107320007A71B0FBF1F717B9012700E00027FCF7ED
:1073300035FE0446B9B26A46DAF80000FCF77AF87E
:1073400080463EB11248804502D10020306001E005
:10735000C6F800809DF800000A2802D14FF0FF34E3
:1073600013E000BF00BFFCF719FE0546A54201D996
:107370002D1B02E0C4F1FF3005444FF47A706843DE
:107380004FF47A71B0FBF1F0441C2046BDE8F88F51
:107390001C01002010B5F8F78BFF10BDF8B50746AB
:1073A0000C464CB14FF47A7060434FF47A71B0FBE5
:1073B000F1F616B9012600E00026FCF7EFFD0446C1
:1073C000B1B26A463868FCF7ABF99DF800000A28AC
:1073D00002D14FF0FF3411E0FCF7E0FD0546A54275
:1073E00001D32D1B02E0C4F1FF3005444FF47A7045
:1073F00068434FF47A71B0FBF1F0441C2046F8BDAD
:1074000010B504462046F8F757FF10BD08B56B4687
:10741000542214210248FBF745FF0249086008BDC9
:10742000000401201401002038B504460D46142D37
:1074300000DD142569460E480068FBF771FF2060E7
:107440009DF8000080B9A9B22268101DFBF7A2FFC9
:10745000216808602068006808B1002038BD214616
:1074600003480068FBF77BFF4FF0FF30F6E70000B2
:107470001401002070B504460D4605B9044D00BF47
:10748000216808682946FCF767F80028F8D170BD24
:107490001C01002070B505460E4606B9064E296847
:1074A00008683146FCF758F804460CB9002070BD56
:1074B0004FF0FF30FBE700001C010020F0B585B065
:1074C0000446256814216846F8F77DFF6946286858
:1074D000FCF77BF80646022E07DABDF80400BDF87B
:1074E0000610884201DA012000E0002007463846F5
:1074F00005B0F0BD38B504460D462846FCF7E6F861
:107500002060206810B94FF0FF3038BD6A4603A1F3
:107510002068FBF7FFFD0020F7E700004C574950BB
:107520002053656D0000000010B504462068FCF78C
:107530006FF910BD2DE9F04385B080460D46164623
:107540001F460C9C4FF0000900BF00BF10A1404631
:10755000F8F750FFB0B9F8F7ABFE814603200021E1
:107560004FF400620E4BCDE90132CDE90310A0B219
:10757000E3B20C4A00902846FCF7C6F94846F8F7F3
:107580009BFE00E00024E0B205B0BDE8F0830000FF
:1075900074637069705F74687265616400000000F4
:1075A000900A01208C2A01202DE9F04106460F4661
:1075B000904640F20F1224A10920FFF701F904467A
:1075C0001CB900BF00BFBDE8F08100202060A760AB
:1075D000C4F80C8066602848006810B9264804602A
:1075E000F1E7254800684068B0420CD9224800689D
:1075F0004068801B2049096848601F480068206077
:107600001D4804601DE01C48056817E06068696853
:10761000401A6060286820B1286840686168884224
:107620000BD9286828B1286840686168401A296821
:107630004860286820602C6002E02D68002DE5D1AC
:1076400000BF00BFBFE700002E2E5C5372635C5585
:1076500073725C4472697665725C557044726976C7
:1076600065725C6C7769705C636F72655C74696D80
:107670006572732E63000000F000002010B5002238
:10768000024941F28830FFF78FFF10BD3D4F0000E7
:107690002DE9F0478046894600BF2248006830B98E
:1076A000002249464046FFF72FFE054637E01D48B9
:1076B0000068406840B11B4800684946426840463F
:1076C000FFF722FE054601E04FF0FF35681CA8B920
:1076D00014480468134920680860A668E7682146D2
:1076E0000920FEF7E7FF46B100210F48FFF756FEDD
:1076F0003846B0470C48FFF717FFCEE70948006847
:107700004068A84207D9074800684068401B0549FF
:107710000968486003E00020024909684860BDE844
:10772000F0870000F0000020880000202DE9F041E3
:1077300006460F461448006808B9BDE8F0811248B3
:10774000046800251BE0A068B04216D1E068B8428A
:1077500013D11DB90C492068086001E02068286039
:10776000206828B120684068616808442168486042
:1077700021460920FEF79EFFDFE725462468002CFE
:10778000E1D100BFD9E70000F00000202DE9FC475F
:1077900004460E4600BF00BF207E0A2808D12146BD
:1077A0001F4801F053F921460220FEF783FF34E021
:1077B000276DD4F82880D4F88C50D4F8109000BFEE
:1077C0002146184801F042F901201749087000BF0E
:1077D000206F10B1206F02F0C0FAE06E10B1E06EC1
:1077E00002F0BBFA606F10B1606F02F0B6FA4EB1F2
:1077F000A08B618B231D2246CDE9001041463846FF
:1078000002F02AFA21460220FEF754FF00BF1DB104
:107810006FF009014846A84700BFBDE8FC8700009B
:10782000C0000020BC000020C800002010B50446A5
:1078300001212046FFF7AAFF10BD000070B50646E3
:1078400040F2035239A10220FEF7BAFF0446002C91
:1078500025D100F0D9FD40F2095234A10220FEF7F3
:10786000AFFF044694B9304600F0A4FD40F20F5239
:107870002EA10220FEF7A4FF04463CB13648B0F822
:10788000B400401E81B23448A0F8B4103CB1324874
:10789000B0F8B400401E81B22F48A0F8B410002CFC
:1078A00041D0A0212046F8F78EFD1834667041F2D1
:1078B000D060A4F84E000020A4F8500042F2382016
:1078C000A082E082002004F80F0CFF2004F80E0CC8
:1078D0004FF40670E0830620A08500202085062056
:1078E0006085C01FA0830120A08600F04DFE0546E4
:1078F0002564A5632563656418480068E06018483E
:10790000007860720020E0711648A06640F6B8303A
:10791000A0674FF4FA60E0670620C4F880000020FA
:1079200084F88600183C204670BD00002E2E5C5363
:1079300072635C5573725C4472697665725C5570F3
:107940004472697665725C6C7769705C636F7265AE
:107950005C7463702E63000004020120B0000020FC
:10796000CA000020E19A000010B50446207E0128DC
:1079700003D0A07F40F01000A0770121204600F046
:1079800001F810BD7CB504460E46002E5BD0207E6B
:10799000042802D0207E072855D1A06F20B9A08DE1
:1079A00042F2382188424ED000BF00BFA08B618BCD
:1079B000CDE90010231D2246A16A206D02F04CF98A
:1079C000204601F01FF800BF00BF5A480068A042DF
:1079D00005D158480068C0685649086018E0554805
:1079E0000068554908600EE053480068C068A0422E
:1079F00004D15149E0680968C86008E04E48006851
:107A0000C0684D4908604C4800680028ECD100BFB0
:107A10000020E06000BF01204849087000BF207EC0
:107A200004280AD10A20207600BF45480068E0609B
:107A30004348046002F092FB03E021460220FEF777
:107A400039FE00207CBD207E082868D2DFE800F0E7
:107A500004343F4F5767675F0025608B30B300BF2A
:107A600038480068A04205D136480068C0683549EA
:107A7000086018E0334800682F4908600EE02E487F
:107A80000068C068A04204D12B49E0680968C8605A
:107A900008E029480068C06827490860264800684F
:107AA0000028ECD100BF0020E06000BF214602208A
:107AB000FEF700FE002435E000252146224800F0B4
:107AC000C5FF21460320FEF7F5FD00242AE000252E
:107AD00000BF2146174800F0B9FF01201749087080
:107AE00000BF21460220FEF7E5FD00241AE02046F3
:107AF00002F066F905460DB90520207612E0204611
:107B000002F05EF905460DB9052020760AE0204610
:107B100002F056F905460DB90920207602E000254D
:107B2000002400BF00BF1CB115B9204600F082FD43
:107B3000284687E7BC000020C4000020C8000020C1
:107B4000C0000020B4000020B80000202DE9F05F44
:107B500007460E4691469A46DDF8288008F0010057
:107B600008B1042000E0002008F0020109B10C2156
:107B700000E000214518A42224A10420FEF720FEE5
:107B8000041E05D13046FFF72DFA0020BDE8F09F16
:107B900084F80A800020206066603089401B2081C4
:107BA00014213046FFF783FA60B12448B0F88C0006
:107BB000401C81B22148A0F88C10204602F0C0F889
:107BC0000020E3E760684068E060788BFEF7E1FA48
:107BD000E1680880B88BFEF7DCFAE168488050461F
:107BE000FEF7CAFAE1684860AB46E91705EB917108
:107BF0008910491D49EA013188B2FEF7CAFAE168E5
:107C000088810020E16848822046BFE72E2E5C5321
:107C100072635C5573725C4472697665725C557010
:107C20004472697665725C6C7769705C636F7265CB
:107C30005C7463705F6F75742E6300000402012032
:107C40002DE9F04105460E463046FEF771F904462F
:107C500054B1A08D40B1A08D283887B2BD4201DA61
:107C6000284600E0384605462846BDE8F081000079
:107C70002DE9F84304460D460027B84600BF00BF73
:107C8000B4F86800102805DAB4F868004FF6FC7103
:107C900088420FD94A48B0F88400401C81B2484855
:107CA000A0F88410A07F40F08000A0774FF0FF3054
:107CB000BDE8F88305F0020000B1012707F00100DC
:107CC00008B1042000E0002007F0020109B10C21F6
:107CD00000E0002100EB0108B4F8660050B9384814
:107CE000B0F88400401C81B23548A0F884104FF0F1
:107CF000FF30DDE7002241461046FEF7B5FFB0F148
:107D000000090ED1A07F40F08000A0772C48B0F889
:107D10008400401C81B22A48A0F884104FF0FF3044
:107D2000C6E700BF00BF00972A4649462046E36DDC
:107D3000FFF70CFF061E0DD1A07F40F08000A0775A
:107D40001F48B0F88400401C81B21D48A0F8841080
:107D5000701EADE700BF00BF00BF00BFE06E08B9F6
:107D6000E66607E0E06E00E0006801680029FBD1EC
:107D7000066000BF0020A4F86A0005F0020010B9F8
:107D800005F0010038B1E06D401CE065B4F8660014
:107D9000401EA4F8660005F0010018B1A07F40F075
:107DA0002000A0777068FFF76BF834F8681F08446C
:107DB000208034F8680908B100BF00BF002077E7D1
:107DC0000402012070B51B480078401C1949087056
:107DD00000BF1948046829E094F821001549097882
:107DE000884223D01348007884F82100A07F00F057
:107DF000010060B100BFA07F40F00200A07700BF8B
:107E0000204600F017FCA07F20F00300A077E56873
:107E1000A06F48B1002009490870204601F026F9FA
:107E20000648007800B1D4E72C4600BF002CD3D11F
:107E300070BD0000CA000020BC000020C800002067
:107E4000704700002DE9FC4706468A46FB48B0F81B
:107E50007A00401C81B2F948A0F87A10F84970689D
:107E60000860F74871680068007800F00F0001EBC7
:107E70008000F4490860F248006800780007800E2E
:107E800041423046FFF713F910B93089142808D25F
:107E9000EA48B0F88200401C81B2E848A0F882109D
:107EA0003BE2E94908685146FDF78DFE28B9E648EE
:107EB000007800F0F000E02808D1E048B0F8880031
:107EC000401C81B2DD48A0F8881026E2DD4909682F
:107ED0008889FEF77EF94FEA20394FEA890041424E
:107EE0003046FFF7E4F840B1D448B0F88200401CB7
:107EF00081B2D248A0F882100FE2D24909680888FE
:107F0000FEF767F9CF4909680880CE4909684888B3
:107F1000FEF75FF9CB4909684880CA490968486893
:107F2000FEF751F9C74909684860C8490860C54962
:107F300009688868FEF747F9C24909688860C4493A
:107F40000860C0490968C889FEF743F9BD49096856
:107F5000C881BC4909688889FEF73BF900F03F00F9
:107F6000BC4908703089097801F0030109B1012189
:107F700000E000210844B84908800027B748046899
:107F80002AE000BF00BF00BF00BF00BF00BFA08B42
:107F9000AC490968098888421CD1608BA9490968E5
:107FA0004988884216D1AE4960680968884211D173
:107FB000A5492068096888420CD100BF00BF37B1CD
:107FC000E068F860A5480068E060A448046000BF6D
:107FD00000BF03E02746E468002CD2D100BF002C8C
:107FE0004DD1A048046820E000BF00BFA08B954998
:107FF00009680988884217D1608B924909684988C5
:10800000884211D196496068096888420CD18E492E
:1080100020680968884207D1204602F0BBF8304644
:10802000FEF7E0FFBDE8FC87E468002CDCD1002708
:108030008D48056810E0688B824909684988884244
:1080400008D1814928680968884202D00DB12868A2
:1080500000B903E02F46ED68002DECD100BF75B1EB
:1080600037B1E868F86080480068E8607E480560DD
:10807000284600F0E7F93046FEF7B4FFD2E7002CBF
:108080007ED0002079490860308908810846466022
:108090006C480068C8600020754908607549087020
:1080A0006C48007800F0080018B1707B40F00100C7
:1080B0007073A06F98B1204600F0D8FF0A3028B145
:1080C000A06F60B164480088002808DD5B48B0F804
:1080D0007E00401C81B25948A0F87E10DDE0664861
:1080E0000460204600F0FCFC804608F10A000028ED
:1080F00017D06048007800F0080098B100BFD4F8AD
:108100008C0028B16FF00A01D4F88C2020699047C8
:1081100000BF2146514800F099FC21460220FEF79D
:10812000C9FAB9E05348007800F01000B8B1A07F58
:1081300000F0100050B900BFD4F88C0028B16FF0E7
:108140000B01D4F88C202069904700BF214643489A
:1081500000F07CFC21460220FEF7ACFA9CE04FF0D8
:108160000008B4F86400002812DD00BFE06F40B1E1
:10817000B4F864202146E36F20699847804602E006
:108180009BE04FF0000800BF08F10A0000B984E04E
:108190003748006870B300BF00BFA07F00F0100038
:1081A00038B133480068FEF71DFF2046FFF73EFB5D
:1081B00073E000BFD4F8800048B100232C49D4F804
:1081C00080C020690A682146E047804607E0002316
:1081D000274821460268184601F082FC804600BF0D
:1081E00008F10A0000B958E0B8F1000F02D02048A9
:1081F0000068A0671F48007800F02000E8B1A06F79
:1082000030B1A06F407B40F02000A16F48733DE08B
:10821000A08D42F23821884202D0A08D401CA0855A
:1082200000BFD4F8800048B300231A462146D4F892
:1082300080C02069E047804623E027E00402012057
:10824000D4000020D00000200C010020D800002025
:10825000DC000020E0000020E2000020BC00002044
:1082600008010020C0000020B800002028030120E1
:10827000E8000020E4000020EC000020FFE74FF0C1
:10828000000800BF08F10A0000B906E000202949F3
:108290000860204600F0CEF900BF002025490860A4
:1082A0002549086025484068A0B324494868FEF77E
:1082B00099FE0020214948602CE0214909688889FD
:1082C000FDF787FF00F0040008BB1E48B0F88800E7
:1082D000401C81B21B48A0F88810B0F87E00401CFA
:1082E00081B21848A0F87E1015480068008814492B
:1082F00009684988CDE9001013480068134A1288BC
:108300008118134B134A1448006801F0A5FC30464D
:10831000FEF768FE00BF00BF84E60A48B0F87E00A2
:10832000401C81B20748A0F87E103046FEF75AFE86
:1083300000BF77E6EC000020E800002028030120C1
:10834000D000002004020120D8000020E20000201C
:10835000080100200C010020DC0000202DE9FC4178
:108360000446216D481EFDF707FF07463B460022E5
:108370001146204600F03EFA05460DB9BDE8FC81E5
:108380006E680B48B0F87800401C0949A1F87800E5
:1083900006200021CDE90010A37A221D214628469F
:1083A000FDF73CFD2846FEF71DFE00BFE6E7000096
:1083B000040201202DE9F04106464FF07F08002716
:1083C00000250F48046813E0607EB0420FDC607E39
:1083D00040450CDC0B49606A0968081AB84206D3AC
:1083E0000849606A09680F1A254694F81980E468FC
:1083F000002CE9D115B12846FFF718FABDE8F08145
:10840000BC000020B000002070B5002600250B48FD
:1084100004680BE00A49606A0968081AB04204D38C
:108420000749606A09680E1A2546E468002CF1D1F4
:1084300015B12846FFF7FAF970BD0000C000002012
:10844000B00000207CB505464548007800F00400E7
:1084500008B100207CBD4248007800F0100098B1BF
:108460004048006800883F4909684988CDE9001004
:108470003D4800683D4A128881183D4B3D4A3E48C0
:10848000006801F0E9FB69E03548007800F002007F
:10849000002863D0687EFFF7D1F9044654B9374805
:1084A000B0F88400401C81B23448A0F884104FF02A
:1084B000FF30CFE72F4800682060688B60832C482E
:1084C00000686060274800680088A0830320207649
:1084D00025480068401CA062A06A2063214800680B
:1084E000C089A4F860001F480068C089A4F8620031
:1084F000B4F86000A4F84E001B480068401E606598
:108500002869206168696061287A00F08C00207217
:1085100000BF00BF1A480068E0601948046001F01D
:108520001DFE00BF01201749087000BF204600F063
:108530000DFAE08E211DFFF783FBE0861221204615
:10854000FFF796FB06462EB100212046FFF71EF9E5
:1085500030467FE7204600F06DF87BE7002079E7A2
:10856000E0000020D0000020D8000020E200002021
:10857000080100200C010020DC0000200402012082
:10858000BC000020C80000200448006804490968B5
:10859000084402490860084600687047CC00002083
:1085A000B000002070B505460C46E9688889FDF7E3
:1085B00010FE00F0010020B1204601F0CEFB0024A7
:1085C00033E013E0E1688889FDF703FE00F0010065
:1085D00038B10120FDF7DDFDE96889890843E968C4
:1085E000888126462468304601F0AAFB4CB1E06839
:1085F00040682189084429890D4A12681144081AE3
:10860000E0D594B128890A4909680844E1684968B5
:10861000401A002809DDE068808805490988401A69
:10862000288129896868FEF7A5FD2C6070BD0000CF
:10863000D80000202DE9F047044600BF00BF6C4879
:108640000068A04202D10020BDE8F087B4F86000C5
:10865000B4F84C10884202DAB4F8600001E0B4F8D3
:108660004C008146E56EA07F00F0020070B14DB174
:10867000E9684868FDF7A7FDA16C401A29890844FC
:10868000484503D9204601F074FBDDE7266F26B18B
:1086900000E0366830680028FBD191E000BFE9684F
:1086A0008889FDF796FD00BF206FA0B1A07F00F084
:1086B000440080B9E06E38B1E06E006858B9E06EF1
:1086C0000089E18E884206DAB4F8660018B1B4F881
:1086D0006800102801DB012000E0002020B9A07F05
:1086E00000F0A00000B977E02868E066207E02284C
:1086F0000BD01020FDF74DFDE96889890843E96832
:108700008881A07F20F00300A0772146284600F052
:10871000ADF8E9684868FDF756FD0746E9688889BD
:10872000FDF757FD00F0030008B1012000E0002034
:108730002989084407EB0008206DB0EB080001D53B
:10874000C4F85080E9688889FDF743FD00F0030014
:1087500008B1012000E000202989084400282BDD11
:1087600000202860206F10B925672E4627E0E968B1
:108770004868FDF728FD0746F1684868FDF723FDC6
:10878000381A16D504F1700700E03F68386860B108
:108790003968C9684868FDF716FD8246E968486887
:1087A000FDF711FDBAEB0000EFD4386828603D609A
:1087B00005E03560366802E0284601F0C1FAE56E52
:1087C00055B1E9684868FDF7FEFCA16C401A29899B
:1087D000084448457FF662AF00BFE06E10B9002044
:1087E000A4F86A00A07F20F08000A07700202BE78B
:1087F000EC0000202DE9F04705460E4690469946CC
:1088000006F11400404481B200220120FEF72CFA48
:10881000074647B300BF00BF7C68688BFDF7B9FC13
:108820002080A88BFDF7B5FC6080C4F80490A86A8E
:10883000FDF7A2FCA060B246F11706EB917189101A
:10884000491D102242EA013188B2FDF7A2FCA08145
:10885000E88DFDF79EFCE081002020826082E98D9A
:10886000A86A084428633846BDE8F0872DE9FC472C
:1088700005460C46A06AFDF77FFCE9688860E08D3C
:10888000FDF787FCE968C881E18DA06A0844206390
:10889000E86800F11408A87A00F0010070B1211D09
:1088A00040F2B450FFF7CCF9814649F00170FDF772
:1088B00063FCC8F8000008F1040800BFB4F93400F4
:1088C000401C08B90020A0860CB1206840B9201DCA
:1088D000FDF72EFB06460EB9BDE8FC8770682060E8
:1088E000A06B38B917480068A063E9684868FDF7CD
:1088F0006AFCE063A88969688988401A87B2686859
:108900004089C01B6968488168680089C01B696824
:1089100008816968E86848600020E96808820A48B8
:10892000B0F87800401C0849A1F878000621607A68
:10893000CDE90001A37A221D21466868FDF76EFA91
:1089400000BFC9E7B0000020040201202DE9F04774
:1089500080462B48006800F1140529490968888978
:10896000FDF737FC0521B1EB203F46DA24490968C1
:108970008889FDF72EFC0521C1EB20304FF6FF71F1
:1089800001EA8006002436E015F80490B9F1000FE2
:1089900006D0B9F1010F05D0B9F1020F21D104E0E1
:1089A000BDE8F087601C84B224E0601C285C0428C9
:1089B00002D1201DB04200DDF2E7E01C295CA01CC2
:1089C000285C41EA002740F2B450874200DC17B926
:1089D00040F2B45000E03846A8F83600201D84B2BA
:1089E00008E0601C285C00B9DAE7601C285C2044C1
:1089F00084B200BF00BFB442C6DB00BFD0E70000B6
:108A0000D000002010B50446207EF0B1207E0A2858
:108A10001BD0207E012818D0A06F20B1A06FFEF7D8
:108A2000E1FA0020A067606F01F097F9002060670D
:108A3000401EA086E06E01F090F9206F01F08DF9E4
:108A40000020E0662067A4F86A0010BD70B50546F6
:108A50000C4600BF2868A04203D12868C06828607F
:108A600017E01E49286808600EE01C480068C068CE
:108A7000A04204D11949E0680968C86008E01748B5
:108A80000068C06815490860144800680028ECD1E7
:108A900000BF0020E06000BF2046FFF7B3FF207E4C
:108AA0000A280DD0207E01280AD0A07F00F0010006
:108AB00030B1A07F40F00200A0772046FFF7BAFD5A
:108AC000207E012805D000BF00BF00BF00BF00BF4F
:108AD00000BF0020207600BF00BF70BDC400002092
:108AE0002DE9FC4104464FF000080026FE480078BE
:108AF00000F0040070B3207E022807D1FB49206DEE
:108B00000968884211D14FF001080EE0F849A06AC7
:108B10000968081A09D4A18DA06A0844F4490968B3
:108B2000081A002801DC4FF00108B8F1000F0FD03F
:108B300000BF00BFEF48007840F00800ED49087022
:108B4000A07F20F00100A0776FF00A00BDE8FC8153
:108B50000020FBE7E448007800F0020068B1207EC6
:108B600002280AD0207E032807D000BFA07F40F053
:108B70000200A07700BF0020E8E7A07F00F010000F
:108B800010B9DD4800686062002084F89E0020462D
:108B9000FFF7DCFE207E801E082873D2DFE800F09D
:108BA000049BF0EFEEEDECEBCF48007800F0100006
:108BB000002877D0CC48007800F00200002871D05F
:108BC000216FC9684868FDF7FEFA401CC74909686B
:108BD000884267D12834E08F401CE087C448006891
:108BE000401C20602068A060C04800682062C34824
:108BF0000068C0892087C1480068C0896087BC4878
:108C00000068401EE062042004F8100CE089283C53
:108C1000211DFFF715F8E086E08E00EB80004FF68F
:108C2000FF7101EA4000A4F84E00B4F84C0001289E
:108C300002D1E08E400000E0E08EA4F84C0000BFBE
:108C400000BFB4F86800401EA4F86800256F2868CB
:108C50002067284601F074F8206F18B94FF0FF30F4
:108C6000A08603E00020A08684F8460000BFD4F868
:108C7000840048B100222146D4F884302069984706
:108C8000064602E0E0E10DE0002600BF06F10A0022
:108C900010B96FF0090059E700BFA07F40F0020053
:108CA000A07717E09048007800F0100090B193484A
:108CB00000680088914909684988CDE900108C480E
:108CC00000688F4A128881188E4B8F4A8748006847
:108CD00000F0C2FFB9E18448007800F010000028DD
:108CE00063D0A06C401C81490968081A49D47F49A7
:108CF000206D0968081A002843DC0420207600BF94
:108D000000BF00BF606930B100222146D4E90403EE
:108D10009847064601E06FF00D0600BF46B106F128
:108D20000A0010B12046FEF781FD6FF009000DE743
:108D3000B4F84C70204600F0E1F9B4F8640020B1BA
:108D4000B4F86400401EA4F86400012F02D1E08E44
:108D5000400000E0E08EA4F84C006648007800F087
:108D6000200038B100BFA07F40F00200A07700BF14
:108D70000720207627E053E108E125E0A1E035E077
:108D800023E05E48006800885C4909684988CDE9AD
:108D90000010574800685A4A12888118594B5A4A9D
:108DA0005248006800F058FF0DE04F48007800F08E
:108DB000020040B1A06A401E4D490968884202D1B4
:108DC000204600F0C7FE40E100BF204600F096F9C3
:108DD0004848007800F0200038B100BFA07F40F084
:108DE0000200A07700BF072020762EE1204600F089
:108DF00085F94048007800F02000E8B33A48007850
:108E000000F01000C8B33949206D0968884242D18A
:108E100000BFA07F40F00200A07700BF2046FFF710
:108E2000F1FD00BF00BF39480068A04205D13748B6
:108E30000068C0683549086018E034480068344963
:108E400008600EE032480068C068A04204D1304992
:108E5000E0680968C86008E02D480068C0682C49CF
:108E600008602B4800680028ECD100BF0020E060BB
:108E700000BF0120274901E016E00CE0087000BFA8
:108E80000A20207600BF24480068E0602248046081
:108E900001F064F914E000BFA07F40F00200A07769
:108EA00000BF082020760BE00F48007800F010008B
:108EB00030B10E49206D0968884201D10620207624
:108EC000C3E0204600F01AF90A48007800F02000BC
:108ED00078B300BFA07F40F00200A07700BF20461B
:108EE000FFF790FD00BF19E0E0000020DC0000204B
:108EF000D8000020E4000020B0000020D0000020B6
:108F0000E2000020080100200C010020BC0000202D
:108F1000C4000020C8000020C000002000BF4C4852
:108F20000068A04206D14A480068C0684849086005
:108F300019E02AE046480068464908600EE04548C6
:108F40000068C068A04204D14249E0680968C8606E
:108F500008E040480068C0683E4908603D48006835
:108F60000028ECD100BF0020E06000BF01203A499A
:108F7000087000BF0A20207600BF38480068E06013
:108F80003648046001F0EAF800BF5EE0204600F0D9
:108F9000B5F83348007800F01000E0B33149206D97
:108FA000096888423BD12046FFF72CFD00BF00BF77
:108FB00027480068A04205D125480068C0682449B8
:108FC000086018E022480068224908600EE0214845
:108FD0000068C068A04204D11E49E0680968C86002
:108FE00008E01C480068C0681A4908601948006811
:108FF0000028ECD100BF0020E06000BF012016492E
:10900000087000BF0A20207600BF14480068E060A6
:109010001248046000E002E001F0A0F800BF14E094
:10902000204600F06BF80E48007800F0100050B1B8
:109030000C49206D0968884205D10B48007840F042
:1090400010000949087000E000BF00BF00207DE566
:10905000BC000020C4000020C8000020C000002088
:10906000E0000020DC000020E40000202DE9F041B9
:109070000446A06F477BA66F0020A06700BFD4F80E
:10908000800040B1002332462146D4F880C02069D8
:10909000E047054606E0002332462146184600F028
:1090A0001FFD054600BF05BB07F0200020B3A08DC3
:1090B00042F23821884202D0A08D401CA08500BF1A
:1090C000D4F8800040B100231A462146D4F880C06D
:1090D0002069E047054600E0002500BF05F10A00D1
:1090E00050B96FF00900BDE8F08105F10A0010B930
:1090F0006FF00900F7E7A6670020F4E72DE9FE4FBF
:1091000004460020009000BF00BFFE48007800F039
:10911000100000287ED0B4F86000A16D08440290D1
:10912000F949606D0968401A15D4F749606D0968FE
:10913000884204D1F549A06D0968401A0BD4F3495F
:10914000A06D0968884231D1F1480068C089B4F83F
:10915000601088422ADDEE480068C089A4F86000EB
:10916000B4F86200EA490968C989884204DAE84823
:109170000068C089A4F86200E34800686065E348BD
:109180000068A065B4F8600048B994F89D0068B91B
:10919000002084F89C00012084F89D0006E094F8EB
:1091A0009D00002802DD002084F89D00D749A06CB6
:1091B0000968081A002848DC0020A4F86400D54893
:1091C000008840BBB4F86010A06D01440298814251
:1091D00035D1B4F93400002831DBCC49A06C0968E2
:1091E00088422CD10120009094F84700401CC0B266
:1091F00094F84710884204DD94F84700401C84F836
:10920000470094F84700032812DDB4F84C00E18EC3
:10921000084401E04AE10AE080B2B4F84C10884208
:109220000DDDB4F84C00E18E0844A4F84C0006E0D3
:1092300094F84700032802D1204600F0B8FC0098BB
:10924000002801D184F84700ADE0A06C401CAF4974
:109250000968081A7ED4AD49206D0968081A0028EB
:1092600078DCA07F00F0040038B1A07F20F004007B
:10927000A077B4F84E00A4F84C0000202834A07762
:10928000608BB4F9181000EBE10000B2A083208CD1
:109290009E490988081AA087E08FA18F0844E087BB
:1092A0000020E07799480068206214F8100C283CF0
:1092B000042824DBB4F84C00B4F84E1088420FDACE
:1092C000B4F84C00E18E084480B2B4F84C108842E7
:1092D00015DDB4F84C00E18E0844A4F84C000EE013
:1092E00034F8361F4943E28A91FBF2F1114488B207
:1092F000E18A363C814201DAA4F84C0000BF26E046
:10930000256F206F0068206700BF6868FDF7B8FD13
:1093100000BFB4F8640058B1E9688889FCF759FFC8
:1093200000F0010020B1B4F86400401EA4F864000D
:109330006868FDF7A5FD34F8681F081A20802846E4
:1093400000F0FEFC34F8680908B100BF00BF206FD0
:10935000D8B100E024E0216FC9684868FCF733FF0A
:109360008346216FC9688889FCF733FF00F003004A
:1093700008B1012000E00020216F09890844584409
:1093800062490968401A0028BADD206F18B94FF009
:10939000FF30A08601E00020A0860020E07702E0F8
:1093A0000020A4F864002BE0E56EE06E0068E06643
:1093B000E06E10B90020A4F86A0000BF6868FDF7ED
:1093C0005FFD00BFB4F8640058B1E9688889FCF714
:1093D00000FF00F0010020B1B4F86400401EA4F8C2
:1093E00064006868FDF74CFD34F8681F081A208097
:1093F000284600F0A5FC34F8680908B100BF00BF9A
:10940000E06EF0B1E16EC9684868FCF7DCFE8346A7
:10941000E16EC9688889FCF7DCFE00F0030008B142
:10942000012000E00020E16E0989084458443749D2
:109430000968081A05D43549206D0968081A0028FA
:10944000B2DDA06B90B33149E06B0968401A2DD5AD
:1094500034F8380F30490988081A0FFA80FAB4F93D
:109460000800AAEBE0000FFA80FA2089504400B20D
:109470002081383CBAF1000F03DACAF100000FFA7C
:1094800080FA3834B4F90A00AAEBA0000FFA80FA87
:109490006089504400B260816089B4F9081000EB23
:1094A000E10000B2A081002044F838091948008882
:1094B00000286EDD207E07286BDA1348A16A006859
:1094C000401C081A66D41048A16A0068114A128824
:1094D0001044401E081A00285CDC0B49A06A096889
:1094E000A0EB01090D48D0F8048000BF00BF00BF09
:1094F00000BF40684089484531DA00BF00BF0748D7
:1095000040680DE0E0000020D8000020DC000020D2
:10951000D0000020E2000020B0000020280301203D
:109520000089A0EB090080B201900BE0B8F80A00B6
:10953000A9EB00090198A8F808000020A8F80A0083
:10954000D8F80080B8F80A004845EFDBC9F1000000
:1095500001B24046FDF7ABFD58B100BF09E0F84944
:109560004868C9F1000109B2FDF7A1FD08B100BFCB
:1095700000BFF3480089218DF24A1288891A401AE7
:10958000EF490881EF49A06A0860ED49C968486061
:109590000BE089E2EB49A06A0968081A05D500BF0B
:1095A000A07F40F00200A07700BFE649A06A0968EA
:1095B000081A6FD4A18DA06A0844401EE1490968C9
:1095C000081A002866DCDF49A06A096888426FD162
:1095D000DB49C9688889FCF7FCFD00F0030008B18D
:1095E000012000E00020D64909890844D6490880B6
:1095F000A08D0988884241DAD149C9688889FCF779
:10960000E8FD00F0010098B1CD49C9688889FCF7F0
:10961000E0FD00F03E0B5846FCF7BBFDC849C968A9
:1096200089894CF2FF0211400843C549C968888105
:10963000A08DC3490881C9688889FCF7CAFD00F07C
:10964000020020B1BE480089401EBD490881BC4AC5
:1096500011895068FDF78EFDB949C9688889FCF702
:10966000B8FD00F0030008B1012000E00020B4497B
:1096700009890844B449088000BF00BF606F002812
:1096800015D0AF49C9688889FCF7A3FD00F0010037
:1096900078B109E004E2D4F874B0606F00686067E4
:1096A000584600F04DFB00BF606F0028F3D172E018
:1096B0000DE1656F2DE0E9688889FCF78AFD00F00F
:1096C000010008B39E49C9688889FCF782FD00F053
:1096D0000200C8B90120FCF75CFD9949C968898975
:1096E00008439749C96888819549C9688889FCF702
:1096F00070FD00F0030008B1012000E00020904957
:1097000009890844904908802F462D68384600F0A2
:1097100017FB55B1E8684068298901448948006809
:10972000894A12881044401AC5D59DB385480068FF
:10973000854909880844E9684968401A002829DDF4
:10974000E86880887F490988401A7D490881C9688E
:109750008889FCF73EFD00F0020020B178480089BE
:10976000401E77490881764A11895068FDF702FD4D
:109770007349C9688889FCF72CFD00F0030008B123
:10978000012000E000206E49098908446E490880E4
:1097900000BF00BF65676B4800686B4909880844D3
:1097A000A06200BF00BFA08D67490988401AA0854C
:1097B000204600F057FD624840680089002806DD19
:1097C0005F4840686149086000205D4948605C4925
:1097D000C9688889FCF7FDFC00F0010028B15C48ED
:1097E000007840F020005A49087055E0666F606FBD
:1097F000C068406853490860F1688889FCF7E9FC53
:1098000000F0030008B1012000E000203189084485
:10981000A16A0844A06200BFF1688889FCF7D9FCFE
:1098200000BFF1688889FCF7D4FC00F0030008B1A0
:10983000012000E0002031890844A18D081AA0858C
:10984000204600F00FFD7068008900280DDD3F48BC
:10985000006828B13D4871680068FDF7F5FA02E03C
:109860003A497068086000207060F1688889FCF7E8
:10987000B0FC00F0010050B13548007840F0200005
:1098800033490870207E042801D1072020763068F3
:109890006067304600F054FA606F28B1606FC068AE
:1098A0004068A16A8842A1D000BFA07F00F00100FB
:1098B00040B1A07F20F00100A077A07F40F002001F
:1098C000A07703E0A07F40F00100A07700E12046F0
:1098D00000F04FFA606F20B9194800F005FA606790
:1098E000F6E00027656FD7E0E86840681549096829
:1098F000884213D112480089298988420DDD104819
:1099000000F0F2F906463EB10FB13E6000E0666736
:1099100029463046FEF746FEC1E0C0E0D7B9E86808
:10992000406808490968081A41D5054800F0DCF983
:10993000064626B1666729463046FEF733FEAEE09E
:1099400028030120D8000020E2000020E8000020C9
:10995000E4000020F8684068401C5E490968081A65
:1099600025D4E8684068401E5A490968081A00284A
:109970001DDC594800F0B8F90646BEB1F8684068E9
:109980003989084453490968401A002809DDF868F4
:10999000808850490988081A388139897868FDF724
:1099A000E9FB3E6029463046FEF7FCFD77E028687B
:1099B000E8BBE868406847490968081A002869DD7B
:1099C000E9688889FCF705FC00F0010000B166E059
:1099D000414800F089F92860286848B3E868406881
:1099E000298908443B490968401A002809DDE868CC
:1099F000808838490988081A288129896868FDF70C
:109A0000B9FBA18DA06A014434480088314A12682C
:109A1000104481423DD22968C9688889FCF7D9FB86
:109A200000F00100B0B12968C968888901E031E01F
:109A30002FE0FCF7CEFB00F03E0B5846FCF7A9FBED
:109A40002968C96889894CF2FF02114008432968D6
:109A5000C9688881208DA18D08441E490988401A53
:109A6000296808812A6811895068FDF783FB2968F5
:109A7000C9688889FCF7ADFB00F0030008B101203C
:109A800000E000202968098908441449088000BFC3
:109A900000BF04E02F462D68002D7FF425AF17E0AE
:109AA000204600F066F913E00A49A06A0968081A1E
:109AB00008D4A18DA06A0844401E06490968081A06
:109AC000002805DD00BFA07F40F00200A07700BFA6
:109AD000BDE8FE8FD800002028030120E20000200E
:109AE0002DE9F04107460D4614461E463CB121893A
:109AF000284600F00CF82046FDF774FA05E026B978
:109B00002846FDF731FFBDE8F0810020FBE770B586
:109B100004460E4600BF00BF00BF00BFA08D30440A
:109B2000A085A08D42F23821884201DD0846A0853B
:109B3000204600F097FB054640F68E00854208DB84
:109B400000BFA07F40F00200A07700BF2046FEF7D4
:109B500071FD70BD2DE9F0410446206F08B9BDE8E4
:109B6000F081256F2868206704F16C0600E03668F4
:109B7000306858B13168C9684868FCF724FB07466B
:109B8000E9684868FCF71FFB381AF0D43068286091
:109B90003560286810B90020A4F86A0094F84600DF
:109BA000401C84F846000020A06300BFD7E710B532
:109BB0000446206F90B3A07F00F0040070BB2046E5
:109BC000FFF7C8FFB4F84C00B4F86010884207DD16
:109BD000B4F8600000EBD0714910A4F84E1006E014
:109BE000B4F84C0000EBD0714910A4F84E10B4F852
:109BF0004E00E18E4900884204DAE08E4004000CF9
:109C0000A4F84E00B4F84E00E18E032202FB0100DE
:109C1000A4F84C00A07F40F00400A07710BD70B500
:109C20000446206F00B970BD256F00E02D682868DC
:109C30000028FBD1E06E2860206FE06600202067DE
:109C400094F84600401C84F846000020A06320469B
:109C5000FEF7F0FC00BFE6E72DE9FC5F81460E460B
:109C600017469846DDE90CAB002214210120FCF7D1
:109C7000FBFF05460DB9BDE8FC9F00BF00BF6C6847
:109C80005046FCF786FA20805846FCF782FA60803E
:109C90004846FCF771FA60603046FCF76DFAA06048
:109CA00045F21400FCF775FAA08143F62200E0812A
:109CB0000020208260820B48B0F87800401C0949DF
:109CC000A1F8780006200021FF234246CDE90010CC
:109CD00039462846FCF7A2F82846FDF783F900BF6D
:109CE000C9E700000402012070B5054640F29D421C
:109CF00008A10420FCF764FD04460CB9002070BDE7
:109D000095E80F0084E80F006068FDF76FFA2046C1
:109D1000F5E700002E2E5C5372635C5573725C4451
:109D200072697665725C55704472697665725C6CB6
:109D30007769705C636F72655C7463702E6300009A
:109D400010B5044644B1606810B16068FDF74AF987
:109D500021460420FCF7AEFC10BD70B5044605E0BA
:109D600025682046FFF7ECFF2C4600BF002CF7D1FA
:109D700070BD2DE9FC4104460027206DFCF7FCF97D
:109D800080464346002239462046FEF733FD05460D
:109D900015B9B81EBDE8FC816E68A07F20F00300F5
:109DA000A0770621607ACDE90001A37A221D214621
:109DB0002846FCF733F82846FDF714F90020E9E7B8
:109DC00070B50446E06ED8B1E56E00E02D682868F5
:109DD0000028FBD1E9688889FCF7FBF900F007004F
:109DE00068B90120FCF7D5F9E96889890843E96871
:109DF0008881A07F40F02000A077002070BD00BFC8
:109E000001212046FDF734FFF8E700002DE9FE4F61
:109E100000200290CA480068401CC9490860C9482F
:109E20000078401CC749087000BF0025C648046878
:109E300058E100BF00BF00BF00BF00BF00BF94F8E3
:109E40002100C0490978884201D1E4684AE1BD484F
:109E5000007884F821000026B146207E022806D131
:109E600094F84600062802D1701CC6B26BE094F844
:109E700046000C2802D1701CC6B264E094F89D0024
:109E800000281BDD14F89C0F401C2070217860789E
:109E90009C3C401EAD4A105C814254DB002084F89B
:109EA0009C0094F89D00072804D294F89D00401C63
:109EB00084F89D00204600F0FDF944E0B4F9340038
:109EC000002803DBA08E401C00B2A086206FD0B318
:109ED000B4F93400B4F94410884234DB207E0228FF
:109EE0000CD040346088B4F9001000EBE100A17997
:109EF000974A515C884000B2A080403C0020A08678
:109F0000B4F84C00B4F86010884202DAB4F84C009F
:109F100001E0B4F8600082464FEA6A00A4F84E00FF
:109F2000B4F84E00E18EB0EB410F06DAE08E4FF64A
:109F3000FF7101EA4000A4F84E00E08EA4F84C0046
:109F40002046FFF76CFE207E06280BD1A07F00F094
:109F5000100038B17A49606A0968081A282801D9BE
:109F6000701CC6B2207A00F00800A8B3207E042836
:109F700002D0207E07282FD12434D4E91C21E06EA2
:109F800001FB02004FF4FA71B0FBF1F054F8241910
:109F90006B4A1268511A884206D2701CC6B209F187
:109FA000010000F0FF0917E094F89E10D4E92402A4
:109FB00001FB02004FF4FA71B0FBF1F0604A616AF4
:109FC0001268511A884207D22046FEF7C7F994F862
:109FD0009E00401C84F89E00606F78B15849606A0A
:109FE0000968081AB4F9441001EB4101B0EB410FC4
:109FF00004D3606FFFF7B1FE00206067207E032866
:10A0000007D14F49606A0968081A282801D9701CCD
:10A01000C6B2207E092807D14949606A0968081A32
:10A02000F02801D9701CC6B2A6B32046FEF7EAFCA0
:10A0300025B100BF00BFE068E86004E000BF00BFDA
:10A040004149E0680860B9F1000F09D0A08B618B2D
:10A05000CDE90010231D2246A16A206DFFF7FCFD0B
:10A06000D4F88C80D4F810B02746E4683946022032
:10A07000FCF720FB00203749087000BFB8F1000F43
:10A0800003D06FF009015846C04700BF314800783F
:10A0900008B1CAE600E024E02546E468E87F401CF9
:10A0A000E877E87F95F8201088421ADB0020E877EF
:10A0B0002849087000BFD5F8880030B12946D5F886
:10A0C000882028699047029001E00020029000BF9C
:10A0D0002048007800B1A8E6029810B92846FEF79B
:10A0E000A9FA00BF002C7FF4A4AE00251A4804682A
:10A0F00022E000BF00BF00261149606A0968081A03
:10A10000F02801D9701CC6B2A6B12046FEF77AFC31
:10A1100025B100BF00BFE068E86004E000BF00BFF9
:10A120000D49E06808602746E46839460220FCF7DC
:10A13000C1FA01E02546E468002CDAD1BDE8FE8FC3
:10A14000B0000020CA000020BC000020FDB40000C8
:10A15000F0B40000C8000020C000002010B509487D
:10A16000006868B90848006810B90848006838B144
:10A1700001200449086000220549FA20FDF714FA7D
:10A1800010BD0000F4000020BC000020C000002032
:10A19000DDA400001CB504462148007800F004004E
:10A1A00008B100201CBD1E48007800F0020008B372
:10A1B0001C49A06A0968081A24D4A18DA06A084421
:10A1C00018490968081A00281CDC1748006800882C
:10A1D000154909684988CDE9001012480068134AFA
:10A1E00012888118124B134A13480068FFF734FD98
:10A1F0000020D7E70A48007800F0010010B10F48AE
:10A200000068606209480088002807DDA07F40F0F0
:10A210000200A0772046FEF70DFAC3E70020C1E751
:10A22000E0000020D8000020D0000020E200002044
:10A23000080100200C010020DC000020B0000020FC
:10A2400010B5FDF7BFFD06480078401CC0B20449B8
:10A25000087000F0010008B1FFF7D8FD10BD000044
:10A26000C900002010B501468B8D886AC218C88EBF
:10A2700041F21C140B6BA04201DD204600E0C88EA9
:10A280001844101A04D4888DC885086B101A10BDA4
:10A290000B6B886AC01A002802DD0020C88506E022
:10A2A0008C6A0B6B181B00BF00BFC88500BF002065
:10A2B000EDE700002DE9FC4705462C6F04B9EC6E74
:10A2C0000CB9BDE8FC87E1688889FBF782FF00F0E4
:10A2D000010018B1208908B9012000E00020804663
:10A2E000B8F1000F01D1012000E000208146E068B4
:10A2F00043684A4600212846FEF77CFA064606B91E
:10A30000DFE77768B8F1000F09D01120FBF741FFB4
:10A31000B9894CF2FF0211400843B8810DE0706822
:10A3200000F1140A616809892289891A8BB2012215
:10A3300051466068FCF70DFE00BF0B48B0F878008E
:10A34000401C0949A1F8780006200021CDE9001041
:10A35000AB7A2A1D29463046FBF760FD3046FCF7F4
:10A3600041FE00BFADE70000040201202DE9F041ED
:10A3700005460E4617461548FDF7A0F8002822D0DE
:10A38000D82213A10720FCF71BFA04461CB94FF092
:10A39000FF30BDE8F08105202070A560E66027B1A0
:10A3A00021460A48FDF766F80BE021460748FDF70D
:10A3B00071F830B121460720FCF77CF94FF0FF30EF
:10A3C000E7E70020E5E76FF00500E2E78400002002
:10A3D0002E2E5C5372635C5573725C4472697665B1
:10A3E000725C55704472697665725C6C7769705CFA
:10A3F0006170695C74637069702E630038B50446DF
:10A400000D46FBF7CCFE0D4804600D480560C821E1
:10A410000C48FDF709F808B100BF00BF01210A4848
:10A42000FDF768F808B100BF00BF04204302002216
:10A430000649009006A0FDF77DF838BD7C0000209D
:10A4400080000020840000208800002015A5000066
:10A4500074637069705F7468726561640000000005
:10A4600070B505460E461148FDF728F810B96FF093
:10A47000050070BDB7220EA10820FCF7A1F9044623
:10A4800014B94FF0FF30F4E701202070A560E660BA
:10A4900021460648FCF7FEFF30B121460820FCF7B4
:10A4A00009F94FF0FF30E4E70020E2E784000020E4
:10A4B0002E2E5C5372635C5573725C4472697665D0
:10A4C000725C55704472697665725C6C7769705C19
:10A4D0006170695C74637069702E630010B5044626
:10A4E000FFF7AEFE0748006810B90748006828B1BA
:10A4F00000220649FA20FDF757F802E0002004493F
:10A50000086010BDBC000020C0000020DDA40000D9
:10A51000F400002008B53A48006820B139480068C6
:10A520003749096888474FF4FA70F9F7FBFC0021B6
:10A530003548FCF733FF61E03348FCF7F5FF694627
:10A540003248FDF7A5F800212F48FCF727FF0098B7
:10A55000007807284ED2DFE800F0040C232B353FAB
:10A560004800009A9268101D009A92681168884706
:10A5700043E00098C06890F8350000F0600028B112
:10A58000009AD2E90201FBF739F904E0009AD2E916
:10A590000201FBF73FFB08200099FCF78BF82CE049
:10A5A000009A9268101D009A92681168884724E00A
:10A5B000009B083307CBFCF7F7FF07200099FCF757
:10A5C00079F81AE0009AD2E90301FDF7AFF8072005
:10A5D0000099FCF76FF810E0009AD2E90210884762
:10A5E00007200099FCF766F807E0009AD2E902100C
:10A5F000884702E000BF00BF00BF00BF9CE700002B
:10A600007C000020800000208800002084000020C2
:10A6100070B505462C4600BF6068B0F1005F03D3FB
:10A620000F496068884215D3298903221046FCF738
:10A630001BFB04464CB129462046FCF72AFC064683
:10A640001EB12046FCF7CEFC00242846FCF7CAFCCD
:10A65000204670BD2468002CDED12846F9E70000B2
:10A660000000072070B504463748FAF7F9FA374872
:10A67000F6F7DAFE3648F6F7D7FE60213548F6F7EA
:10A68000FBFE062084F82E0004F12F020021324840
:10A69000F6F72EFC40F2DC50A085322084F835001D
:10A6A000F6F7C6FF122200212B48F6F775FD054686
:10A6B000132200212848F6F76FFD054611220021DC
:10A6C0002548F6F769FD054645F003052B4611229E
:10A6D00000212148F6F779FD3C23122200211E4873
:10A6E000F6F773FD122200211B48F6F755FD0546CB
:10A6F0004FF482611848F6F765FC00211648F6F71A
:10A70000FBFC064631461448F6F7B8FC1248F6F74B
:10A71000A0FD1148F6F787FD10490F48F6F7CBFC6E
:10A720003820F7F72BF8F7F763F80D492820F6F7EC
:10A73000C3F92820F5F756FF4FF490530022114635
:10A740000548F6F742FD70BD090800F0051809003C
:10A75000051409000010064000C00E40C30100802F
:10A76000955F000010B5044600BF00BF0A48A06214
:10A77000742084F83600692137200155074860614C
:10A780000748A06104F12F00034908602046FFF745
:10A7900069FF002010BD000040010020455200006C
:10A7A00065AB000070B505460C46AE6A04F4803017
:10A7B00020B110480068401C0E49086004F40040B5
:10A7C00020B10D480068401C0B49086004F00040AF
:10A7D00010B1284600F012F804F0010010B1304624
:10A7E00000F068F804F4E07010B1284600F0A6F814
:10A7F00070BD00004C01002050010020FEB5054650
:10A80000122200212748F6F7C7FC06461022002135
:10A810002448F6F7C1FC0446012200212148F6F73E
:10A82000BBFC074600BF06F4005098B104F00100DD
:10A8300040B101201C490870012229461B48FFF73E
:10A8400095FD07E0002018490870012229461848A4
:10A85000FFF78CFD06F4A05018B36B4601AA02A9BD
:10A860001048F6F775FB04F0020020B1029820F4BE
:10A870008040029003E0029840F48040029004F08F
:10A88000040020B1029840F40060029003E00298B6
:10A8900020F4006002900348DDE900320299F6F7E7
:10A8A00077FBFEBD00C00E4054010020D36B0000BA
:10A8B000A96B000070B505466C68002639E0A168F8
:10A8C00001EBC101206850F8210000F0004000B108
:10A8D00032E0A16801EBC101206800EB8100006A51
:10A8E000E0B1A16801EBC101206800EB810090F8A4
:10A8F000200000F0010040B9A26802EBC20221680A
:10A9000001EB8201086AFCF76DFB0020A26802EBF4
:10A91000C202216801EB8201086200E00CE0A0683D
:10A92000401CA060D4E90110884201D10020A06041
:10A93000761C6068B042C2D800BF70BD2DE9F041FE
:10A940000546AE6AB468A06810B1A068401E01E078
:10A950006068401E0746FAE0A16801EBC10120686B
:10A9600000EB8100006A002870D0A16801EBC101F2
:10A97000206850F8210000F0004000B1EBE0A16831
:10A9800001EBC101206850F8210000F48070F8B19B
:10A99000A16801EBC101206850F82100C0F30D400F
:10A9A000A26802EBC202216801EB8201096A4881B8
:10A9B000A16801EBC101206800EB8100006A4089B9
:10A9C000A26802EBC202216801EB8201096A0881D8
:10A9D0006248006898B1A26802EBC202206800EBEE
:10A9E0008200016A5D480068FCF72EFA5B48006847
:10A9F000A26802EBC202216801EB82010862A16831
:10AA000001EBC101206800EB8100006A5349086036
:10AA1000A16801EBC101206850F8210000F48070AA
:10AA2000A0B1A16801EBC101206850F8210000F439
:10AA3000004060B149480068FCF7D4FA4848C08833
:10AA4000401C4749C8800020444908601AE0444837
:10AA50004088401C42494880294640480068FFF72A
:10AA6000FFFC60B13D480068FCF7BCFA3C488089B7
:10AA7000401C3B4988810846C088401CC880002093
:10AA800036490860032240F2EC511046FCF7ECF81E
:10AA9000A26802EBC202216801EB820108624FF456
:10AAA0008040A26802EBC202216801EB820148608B
:10AAB000A16801EBC101206800EB8100006A70B35E
:10AAC000A16801EBC101206800EB8100006A4068C9
:10AAD000A26802EBC202216801EB82018860A168D2
:10AAE00001EBC101206800EB81004068A26802EB25
:10AAF000C202216801EB8201096A49890843A26800
:10AB000002EBC202216801EB820148604FF0004075
:10AB1000A26802EBC202216841F822000EE0FFE7C2
:10AB20000020A26802EBC202216801EB820188606A
:10AB30000B488089401C0A4988810CE0A068401CB1
:10AB4000A060D4E90110884201D10020A060A06873
:10AB5000B8427FF401AF00BFBDE8F081580100208A
:10AB6000040201202DE9F84F81460E460020009096
:10AB7000FCF710FC00903046FCF738FB3046FFF73E
:10AB800047FD06465EB94E488089401C4C49888185
:10AB90000098FCF735FC4FF0FF30BDE8F88FD9F88E
:10ABA0002840606800686168C96801EBC10100EB7A
:10ABB0008105286A68B13046FCF714FA404880895C
:10ABC000401C3F4988810098FCF71AFC4FF0FF3089
:10ABD000E3E73046FCF754F907466068806861682F
:10ABE000C968884205D9606880686168C968401A88
:10ABF00006E06068C068C0F11800616889680844B0
:10AC00008346BB450DD23046FCF7ECF92C488089D1
:10AC1000401C2B4988810098FCF7F2FB4FF0FF3075
:10AC2000BBE74FF0010A4FF080502860B04638E093
:10AC3000606800686168C96801EBC10100EB8105CB
:10AC4000B8F80A006860D8F80400A860BAF1000FEC
:10AC500005D04FF0000A4FF08050286001E000203E
:10AC60002860286840F4500028607F1ED8F80080D3
:10AC70006068C068401C6168C8606068C068182867
:10AC800002D100206168C8602FB9286840F0C04038
:10AC900028602E6201E0701C2862286840F00040A5
:10ACA0002860002FC4D10748F6F7CFFA044800887F
:10ACB000401C034908800098FCF7A2FB00206CE7C9
:10ACC0000402012000C00E40704700002DE9FF5F24
:10ACD00005460E467B48B0F86200401C81B27948B8
:10ACE000A0F86210D5F804B029899BF8000000F0A4
:10ACF0000F00082202EB8000814208DB9BF8000075
:10AD00000007800E41422846FCF7D1F990B16D480A
:10AD1000B0F86A00401C81B26A48A0F86A10B0F826
:10AD20006600401C81B26748A0F866102846FCF710
:10AD300059F9C4E0D5F80490634908683146FAF738
:10AD400042FF8046B9F80000FBF743FA0390B9F8D8
:10AD50000200FBF73EFA0290002700200190824695
:10AD60005A4804684CE000200190618A02988142B0
:10AD700023D1B8F1000F02D1ACB1206898B152498B
:10AD80002068096888420ED0B8F1000F15D054B180
:10AD9000206840B12168B06801404B480068B26843
:10ADA0001040814209D101200190BAF1000F04D175
:10ADB000207C00F0040000B9A2460198F0B1A18AFD
:10ADC000039881421AD1201D30B1606820B14049FA
:10ADD00060680968884211D13FB1E068F8603B487B
:10ADE0000068E0603948046007E03648B0F8760053
:10ADF000401C81B23348A0F8761003E02746E4688F
:10AE0000002CB0D100BF04B9544624B92E49706853
:10AE1000096888424FD16FF007012846FCF747F9CF
:10AE200068B100BF00BF2748B0F86600401C81B27F
:10AE30002448A0F866102846FCF7D4F83FE074B127
:10AE4000A06940B103980090214B2A462146D4E9DD
:10AE500006C0E04732E02846FCF7C4F82FE0B8F11E
:10AE6000000F15D11848007800F0F000E0280FD04E
:10AE70009BF8000000F00F00082202EB800128463A
:10AE8000FCF715F900BF00BF03212846FAF72AFD99
:10AE90000C48B0F87000401C81B20A48A0F870104D
:10AEA000B0F86600401C81B20648A0F8661028463B
:10AEB000FCF798F802E02846FCF794F800BFBDE8DC
:10AEC000FF9F0000040201200C010020FC00002074
:10AED000080100200090D0030C00000000EA3206B8
:10AEE0000000000080D1F008040000000040004095
:10AEF00010000000008005401000000000500040DD
:10AF000011000000009005401100000000600040AA
:10AF10001200000000A00540120000000070004078
:10AF20001300000000B00540130000000040024084
:10AF30001400000000C00540140000000050024052
:10AF40002E00000000D005402E00000000600240EE
:10AF50002F00000000E005402F00000000700240BC
:10AF60003000000000F005403000000000D0034039
:10AF700046000000000006404600000000100640A9
:10AF80004700000000200640480000000030064056
:10AF90007F00000000400640800000000050064096
:10AFA00084000000006006408C000000004000406B
:10AFB000100000000080054010000000005000401C
:10AFC00011000000009005401100000000600040EA
:10AFD0001200000000A005401200000000700040B8
:10AFE0001300000000B005401300000000400240C4
:10AFF0001400000000C00540140000000050024092
:10B000002E00000000D005402E000000006002402D
:10B010002F00000000E005402F00000000700240FB
:10B020003000000000F005403000000000D0034078
:10B0300043000000000006404300000000100640EE
:10B04000440000000020064045000000003006409B
:10B050005800000000400640590000000050064023
:10B060005C000000006006406400000000700640C4
:10B070006C000000008006406D000000009006405B
:10B080007F0000000040004000800540005000406C
:10B09000009005400060004000A0054000700040A6
:10B0A00000B005400040024000C005400050024092
:10B0B00000D005400060024000E005400070024002
:10B0C00000F0054000D0034000000640001006409C
:10B0D00000100640002006400020064000300640D8
:10B0E0000030064000400640004006400050064048
:10B0F00000500640006006400060064000700640B8
:10B100000070064000800640008006400090064027
:10B110000090064000070000000600000005000047
:10B120000004000000030000000200000001000015
:10B13000000000000000000018ED00E01CED00E041
:10B1400020ED00E000E400E004E400E008E400E0BA
:10B150000CE400E010E400E014E400E018E400E097
:10B160001CE400E020E400E024E400E028E400E047
:10B170002CE400E030E400E034E400E038E400E0F7
:10B180003CE400E040E400E044E400E048E400E0A7
:10B190004CE400E050E400E054E400E058E400E057
:10B1A0005CE400E060E400E064E400E068E400E007
:10B1B0006CE400E070E400E074E400E078E400E0B7
:10B1C0007CE400E080E400E084E400E088E400E067
:10B1D00000E100E004E100E008E100E00CE100E053
:10B1E00010E100E080E100E084E100E088E100E0BF
:10B1F0008CE100E090E100E000E200E004E200E029
:10B2000008E200E00CE200E010E200E080E200E092
:10B2100084E200E088E200E08CE200E090E200E0FE
:10B22000010000007856341201003F0001001800B0
:10B23000E805010001001000140002000A000100EE
:10B240003F00010001000A0001001800F0000100A9
:10B25000040001000A0018000800010004000100B9
:10B2600001000100800001003400010001008000A5
:10B2700001000100010040005800E80301001A72BB
:10B280000100100001000800E80328008002080007
:10B2900040006224000001000200010003000100E0
:10B2A000020001000400010002000100030001008F
:10B2B000020001000500010002000100030001007E
:10B2C000020001000400010002000100030001006F
:10B2D000020001000600010002000100030001005D
:10B2E000020001000400010002000100030001004F
:10B2F000020001000500010002000100030001003E
:10B30000020001000400010002000100030001002E
:10B31000020001000700010002000100030001001B
:10B32000020001000400010002000100030001000E
:10B3300002000100050001000200010003000100FD
:10B3400002000100040001000200010003000100EE
:10B3500002000100060001000200010003000100DC
:10B3600002000100040001000200010003000100CE
:10B3700002000100050001000200010003000100BD
:10B3800002000100040001000200010003000100AE
:10B39000020001001C002000A0001C001000100092
:10B3A000300014001400100030001C0604000400DB
:10B3B0000700040014000A00080008001000100034
:10B3C000300014006465746563746564206D656D98
:10B3D00070206F766572666C6F7720696E20706F73
:10B3E0006F6C200000000000000000000000000062
:10B3F000000000000000000000000000000000004D
:10B40000000000000000000000000000000000003C
:10B41000000000000000000000000000000000002C
:10B42000000000000000000000000000000000001C
:10B43000000000000000000000000000000000000C
:10B44000000000006465746563746564206D656D5B
:10B450007020756E646572666C6F7720696E2070FF
:10B460006F6F6C2000000000000000000000000072
:10B4700000000000000000000000000000000000CC
:10B4800000000000000000000000000000000000BC
:10B4900000000000000000000000000000000000AC
:10B4A000000000000000000000000000000000009C
:10B4B000000000000000000000000000000000008C
:10B4C0000000000044B500006CB500008CB5000021
:10B4D0004CB5000038B5000020B500002CB50000C8
:10B4E00080B5000058B5000060B5000074B50000DC
:10B4F0000102030405060707070707070703060CF1
:10B5000018306078B8000020B4000020BC00002093
:10B51000C0000020FFFFFFFFFFFF00000000000051
:10B5200046494E5F574149545F31000046494E5FDE
:10B53000574149545F32000045535441424C4953EE
:10B5400048454400434C4F534544000053594E5F17
:10B550005243564400000000434C4F53494E4700AD
:10B560004C4153545F41434B000000004C4953543D
:10B57000454E000054494D455F5741495400000075
:10B58000434C4F53455F57414954000053594E5F58
:10B5900053454E5400000000B8B5000000000020E4
:10B5A0009001000050040000ECB500009001002064
:10B5B00078DD01002C4F000001AD021EC00B486E6B
:10B5C000194C1AFF01131801B720BC2A012018F6E4
:10B5D0001C2E0120081A20281A3004092BCB1CA885
:0CB5E0000CF063290842FE637A040000AE
:0400000500000201F4
:00000001FF
